 windowsaccessbridge

 Timestamp is 1fb96336 (reproducible build file hash)

 Preferred load address is 10000000

 Start         Length     Name                   Class
 0001:00000000 00006644H .text$mn                CODE
 0002:00000000 00000108H .idata$5                DATA
 0002:00000108 00000008H .00cfg                  DATA
 0002:00000110 00000004H .CRT$XCA                DATA
 0002:00000114 00000004H .CRT$XCZ                DATA
 0002:00000118 00000004H .CRT$XIA                DATA
 0002:0000011c 00000004H .CRT$XIZ                DATA
 0002:00000120 00000004H .CRT$XPA                DATA
 0002:00000124 00000004H .CRT$XPZ                DATA
 0002:00000128 00000004H .CRT$XTA                DATA
 0002:0000012c 00000004H .CRT$XTZ                DATA
 0002:00000130 00000000H .gfids$y                DATA
 0002:00000130 00003390H .rdata                  DATA
 0002:000034c0 00000000H .rdata$CastGuardVftablesA DATA
 0002:000034c0 00000000H .rdata$CastGuardVftablesC DATA
 0002:000034c0 0000012cH .rdata$r                DATA
 0002:000035ec 00000004H .rdata$sxdata           DATA
 0002:000035f0 0000006cH .rdata$voltmd           DATA
 0002:0000365c 000002e0H .rdata$zzzdbg           DATA
 0002:0000393c 00000004H .rtc$IAA                DATA
 0002:00003940 00000004H .rtc$IZZ                DATA
 0002:00003944 00000004H .rtc$TAA                DATA
 0002:00003948 00000008H .rtc$TZZ                DATA
 0002:00003950 00000120H .xdata$x                DATA
 0002:00003a70 00000e40H .edata                  DATA
 0002:000048b0 000000a0H .idata$2                DATA
 0002:00004950 00000014H .idata$3                DATA
 0002:00004964 00000108H .idata$4                DATA
 0002:00004a6c 0000051cH .idata$6                DATA
 0003:00000000 00000028H .data                   DATA
 0003:00000028 00000060H .data$r                 DATA
 0003:00000088 00000018H .data$rs                DATA
 0003:000000a0 000003a4H .bss                    DATA
 0004:00000000 00000120H .rsrc$01                DATA
 0004:00000120 00000640H .rsrc$02                DATA

  Address         Publics by Value              Rva+Base       Lib:Object

 0000:00000000       ___AbsoluteZero            00000000     <absolute>
 0000:00000000       ___arm64x_extra_rfe_table  00000000     <absolute>
 0000:00000000       ___arm64x_extra_rfe_table_size 00000000     <absolute>
 0000:00000000       ___arm64x_native_entrypoint 00000000     <absolute>
 0000:00000000       ___arm64x_redirection_metadata 00000000     <absolute>
 0000:00000000       ___arm64x_redirection_metadata_count 00000000     <absolute>
 0000:00000000       ___dynamic_value_reloc_table 00000000     <absolute>
 0000:00000000       ___enclave_config          00000000     <absolute>
 0000:00000000       ___guard_check_icall_a64n_fptr 00000000     <absolute>
 0000:00000000       ___guard_eh_cont_count     00000000     <absolute>
 0000:00000000       ___guard_eh_cont_table     00000000     <absolute>
 0000:00000000       ___guard_fids_count        00000000     <absolute>
 0000:00000000       ___guard_fids_table        00000000     <absolute>
 0000:00000000       ___guard_iat_count         00000000     <absolute>
 0000:00000000       ___guard_iat_table         00000000     <absolute>
 0000:00000000       ___guard_longjmp_count     00000000     <absolute>
 0000:00000000       ___guard_longjmp_table     00000000     <absolute>
 0000:00000000       ___hybrid_auxiliary_delayload_iat 00000000     <absolute>
 0000:00000000       ___hybrid_auxiliary_delayload_iat_copy 00000000     <absolute>
 0000:00000000       ___hybrid_auxiliary_iat    00000000     <absolute>
 0000:00000000       ___hybrid_auxiliary_iat_copy 00000000     <absolute>
 0000:00000000       ___hybrid_code_map         00000000     <absolute>
 0000:00000000       ___hybrid_code_map_count   00000000     <absolute>
 0000:00000000       ___hybrid_image_info_bitfield 00000000     <absolute>
 0000:00000000       ___x64_code_ranges_to_entry_points 00000000     <absolute>
 0000:00000000       ___x64_code_ranges_to_entry_points_count 00000000     <absolute>
 0000:00000001       ___safe_se_handler_count   00000001     <absolute>
 0000:00000100       ___guard_flags             00000100     <absolute>
 0000:00000000       ___ImageBase               10000000     <linker-defined>
 0001:00000000       _PrintDebugString          10001000 f   AccessBridgeDebug.obj
 0001:0000004a       ___local_stdio_printf_options 1000104a f i AccessBridgeDebug.obj
 0001:00000050       __vfprintf_l               10001050 f i AccessBridgeDebug.obj
 0001:00000074       _finalizeFileLogger        10001074 f   AccessBridgeDebug.obj
 0001:0000008d       _fprintf                   1000108d f i AccessBridgeDebug.obj
 0001:000000a5       _getTimeStamp              100010a5 f   AccessBridgeDebug.obj
 0001:000000d3       _initializeFileLogger      100010d3 f   AccessBridgeDebug.obj
 0001:00000195       _printf                    10001195 f i AccessBridgeDebug.obj
 0001:000001b3       ??0AccessBridgeEventHandler@@QAE@XZ 100011b3 f   AccessBridgeEventHandler.obj
 0001:0000020e       ??1AccessBridgeEventHandler@@QAE@XZ 1000120e f   AccessBridgeEventHandler.obj
 0001:0000020e       ??1AccessBridgeMessageQueue@@QAE@XZ 1000120e f   AccessBridgeMessageQueue.obj
 0001:0000020e       @_guard_check_icall_nop@4  1000120e f   MSVCRT:guard_support.obj
 0001:00000211       ?fireCaretUpdate@AccessBridgeEventHandler@@QAEXJPAV_jobject@@0@Z 10001211 f   AccessBridgeEventHandler.obj
 0001:0000022c       ?fireFocusGained@AccessBridgeEventHandler@@QAEXJPAV_jobject@@0@Z 1000122c f   AccessBridgeEventHandler.obj
 0001:00000247       ?fireFocusLost@AccessBridgeEventHandler@@QAEXJPAV_jobject@@0@Z 10001247 f   AccessBridgeEventHandler.obj
 0001:00000262       ?fireJavaShutdown@AccessBridgeEventHandler@@QAEXJ@Z 10001262 f   AccessBridgeEventHandler.obj
 0001:00000273       ?fireMenuCanceled@AccessBridgeEventHandler@@QAEXJPAV_jobject@@0@Z 10001273 f   AccessBridgeEventHandler.obj
 0001:0000028e       ?fireMenuDeselected@AccessBridgeEventHandler@@QAEXJPAV_jobject@@0@Z 1000128e f   AccessBridgeEventHandler.obj
 0001:000002a9       ?fireMenuSelected@AccessBridgeEventHandler@@QAEXJPAV_jobject@@0@Z 100012a9 f   AccessBridgeEventHandler.obj
 0001:000002c4       ?fireMouseClicked@AccessBridgeEventHandler@@QAEXJPAV_jobject@@0@Z 100012c4 f   AccessBridgeEventHandler.obj
 0001:000002df       ?fireMouseEntered@AccessBridgeEventHandler@@QAEXJPAV_jobject@@0@Z 100012df f   AccessBridgeEventHandler.obj
 0001:000002fa       ?fireMouseExited@AccessBridgeEventHandler@@QAEXJPAV_jobject@@0@Z 100012fa f   AccessBridgeEventHandler.obj
 0001:00000315       ?fireMousePressed@AccessBridgeEventHandler@@QAEXJPAV_jobject@@0@Z 10001315 f   AccessBridgeEventHandler.obj
 0001:00000330       ?fireMouseReleased@AccessBridgeEventHandler@@QAEXJPAV_jobject@@0@Z 10001330 f   AccessBridgeEventHandler.obj
 0001:0000034b       ?firePopupMenuCanceled@AccessBridgeEventHandler@@QAEXJPAV_jobject@@0@Z 1000134b f   AccessBridgeEventHandler.obj
 0001:00000366       ?firePopupMenuWillBecomeInvisible@AccessBridgeEventHandler@@QAEXJPAV_jobject@@0@Z 10001366 f   AccessBridgeEventHandler.obj
 0001:00000381       ?firePopupMenuWillBecomeVisible@AccessBridgeEventHandler@@QAEXJPAV_jobject@@0@Z 10001381 f   AccessBridgeEventHandler.obj
 0001:0000039c       ?firePropertyActiveDescendentChange@AccessBridgeEventHandler@@QAEXJPAV_jobject@@000@Z 1000139c f   AccessBridgeEventHandler.obj
 0001:000003be       ?firePropertyCaretChange@AccessBridgeEventHandler@@QAEXJPAV_jobject@@0HH@Z 100013be f   AccessBridgeEventHandler.obj
 0001:000003e0       ?firePropertyChildChange@AccessBridgeEventHandler@@QAEXJPAV_jobject@@000@Z 100013e0 f   AccessBridgeEventHandler.obj
 0001:00000402       ?firePropertyDescriptionChange@AccessBridgeEventHandler@@QAEXJPAV_jobject@@0PAG1@Z 10001402 f   AccessBridgeEventHandler.obj
 0001:00000424       ?firePropertyNameChange@AccessBridgeEventHandler@@QAEXJPAV_jobject@@0PAG1@Z 10001424 f   AccessBridgeEventHandler.obj
 0001:00000446       ?firePropertySelectionChange@AccessBridgeEventHandler@@QAEXJPAV_jobject@@0@Z 10001446 f   AccessBridgeEventHandler.obj
 0001:00000461       ?firePropertyStateChange@AccessBridgeEventHandler@@QAEXJPAV_jobject@@0PAG1@Z 10001461 f   AccessBridgeEventHandler.obj
 0001:00000483       ?firePropertyTableModelChange@AccessBridgeEventHandler@@QAEXJPAV_jobject@@0PAG1@Z 10001483 f   AccessBridgeEventHandler.obj
 0001:000004a5       ?firePropertyTextChange@AccessBridgeEventHandler@@QAEXJPAV_jobject@@0@Z 100014a5 f   AccessBridgeEventHandler.obj
 0001:000004c0       ?firePropertyValueChange@AccessBridgeEventHandler@@QAEXJPAV_jobject@@0PAG1@Z 100014c0 f   AccessBridgeEventHandler.obj
 0001:000004e2       ?firePropertyVisibleDataChange@AccessBridgeEventHandler@@QAEXJPAV_jobject@@0@Z 100014e2 f   AccessBridgeEventHandler.obj
 0001:000004fd       ?setCaretUpdateFP@AccessBridgeEventHandler@@QAEXP6AXJPAV_jobject@@0@ZPAVWinAccessBridge@@@Z 100014fd f   AccessBridgeEventHandler.obj
 0001:0000052f       ?setFocusGainedFP@AccessBridgeEventHandler@@QAEXP6AXJPAV_jobject@@0@ZPAVWinAccessBridge@@@Z 1000152f f   AccessBridgeEventHandler.obj
 0001:00000561       ?setFocusLostFP@AccessBridgeEventHandler@@QAEXP6AXJPAV_jobject@@0@ZPAVWinAccessBridge@@@Z 10001561 f   AccessBridgeEventHandler.obj
 0001:00000593       ?setJavaShutdownFP@AccessBridgeEventHandler@@QAEXP6AXJ@ZPAVWinAccessBridge@@@Z 10001593 f   AccessBridgeEventHandler.obj
 0001:000005d0       ?setMenuCanceledFP@AccessBridgeEventHandler@@QAEXP6AXJPAV_jobject@@0@ZPAVWinAccessBridge@@@Z 100015d0 f   AccessBridgeEventHandler.obj
 0001:0000060d       ?setMenuDeselectedFP@AccessBridgeEventHandler@@QAEXP6AXJPAV_jobject@@0@ZPAVWinAccessBridge@@@Z 1000160d f   AccessBridgeEventHandler.obj
 0001:0000064a       ?setMenuSelectedFP@AccessBridgeEventHandler@@QAEXP6AXJPAV_jobject@@0@ZPAVWinAccessBridge@@@Z 1000164a f   AccessBridgeEventHandler.obj
 0001:00000687       ?setMouseClickedFP@AccessBridgeEventHandler@@QAEXP6AXJPAV_jobject@@0@ZPAVWinAccessBridge@@@Z 10001687 f   AccessBridgeEventHandler.obj
 0001:000006b9       ?setMouseEnteredFP@AccessBridgeEventHandler@@QAEXP6AXJPAV_jobject@@0@ZPAVWinAccessBridge@@@Z 100016b9 f   AccessBridgeEventHandler.obj
 0001:000006eb       ?setMouseExitedFP@AccessBridgeEventHandler@@QAEXP6AXJPAV_jobject@@0@ZPAVWinAccessBridge@@@Z 100016eb f   AccessBridgeEventHandler.obj
 0001:0000071d       ?setMousePressedFP@AccessBridgeEventHandler@@QAEXP6AXJPAV_jobject@@0@ZPAVWinAccessBridge@@@Z 1000171d f   AccessBridgeEventHandler.obj
 0001:0000075a       ?setMouseReleasedFP@AccessBridgeEventHandler@@QAEXP6AXJPAV_jobject@@0@ZPAVWinAccessBridge@@@Z 1000175a f   AccessBridgeEventHandler.obj
 0001:00000797       ?setPopupMenuCanceledFP@AccessBridgeEventHandler@@QAEXP6AXJPAV_jobject@@0@ZPAVWinAccessBridge@@@Z 10001797 f   AccessBridgeEventHandler.obj
 0001:000007d4       ?setPopupMenuWillBecomeInvisibleFP@AccessBridgeEventHandler@@QAEXP6AXJPAV_jobject@@0@ZPAVWinAccessBridge@@@Z 100017d4 f   AccessBridgeEventHandler.obj
 0001:00000811       ?setPopupMenuWillBecomeVisibleFP@AccessBridgeEventHandler@@QAEXP6AXJPAV_jobject@@0@ZPAVWinAccessBridge@@@Z 10001811 f   AccessBridgeEventHandler.obj
 0001:0000084e       ?setPropertyActiveDescendentChangeFP@AccessBridgeEventHandler@@QAEXP6AXJPAV_jobject@@000@ZPAVWinAccessBridge@@@Z 1000184e f   AccessBridgeEventHandler.obj
 0001:0000088e       ?setPropertyCaretChangeFP@AccessBridgeEventHandler@@QAEXP6AXJPAV_jobject@@0HH@ZPAVWinAccessBridge@@@Z 1000188e f   AccessBridgeEventHandler.obj
 0001:000008c3       ?setPropertyChangeFP@AccessBridgeEventHandler@@QAEXP6AXJPAV_jobject@@0PAG11@ZPAVWinAccessBridge@@@Z 100018c3 f   AccessBridgeEventHandler.obj
 0001:000008f5       ?setPropertyChildChangeFP@AccessBridgeEventHandler@@QAEXP6AXJPAV_jobject@@000@ZPAVWinAccessBridge@@@Z 100018f5 f   AccessBridgeEventHandler.obj
 0001:00000935       ?setPropertyDescriptionChangeFP@AccessBridgeEventHandler@@QAEXP6AXJPAV_jobject@@0PAG1@ZPAVWinAccessBridge@@@Z 10001935 f   AccessBridgeEventHandler.obj
 0001:0000096a       ?setPropertyNameChangeFP@AccessBridgeEventHandler@@QAEXP6AXJPAV_jobject@@0PAG1@ZPAVWinAccessBridge@@@Z 1000196a f   AccessBridgeEventHandler.obj
 0001:0000099f       ?setPropertySelectionChangeFP@AccessBridgeEventHandler@@QAEXP6AXJPAV_jobject@@0@ZPAVWinAccessBridge@@@Z 1000199f f   AccessBridgeEventHandler.obj
 0001:000009d4       ?setPropertyStateChangeFP@AccessBridgeEventHandler@@QAEXP6AXJPAV_jobject@@0PAG1@ZPAVWinAccessBridge@@@Z 100019d4 f   AccessBridgeEventHandler.obj
 0001:00000a09       ?setPropertyTableModelChangeFP@AccessBridgeEventHandler@@QAEXP6AXJPAV_jobject@@0PAG1@ZPAVWinAccessBridge@@@Z 10001a09 f   AccessBridgeEventHandler.obj
 0001:00000a49       ?setPropertyTextChangeFP@AccessBridgeEventHandler@@QAEXP6AXJPAV_jobject@@0@ZPAVWinAccessBridge@@@Z 10001a49 f   AccessBridgeEventHandler.obj
 0001:00000a7e       ?setPropertyValueChangeFP@AccessBridgeEventHandler@@QAEXP6AXJPAV_jobject@@0PAG1@ZPAVWinAccessBridge@@@Z 10001a7e f   AccessBridgeEventHandler.obj
 0001:00000ab3       ?setPropertyVisibleDataChangeFP@AccessBridgeEventHandler@@QAEXP6AXJPAV_jobject@@0@ZPAVWinAccessBridge@@@Z 10001ab3 f   AccessBridgeEventHandler.obj
 0001:00000af3       ??0AccessBridgeJavaVMInstance@@QAE@PAUHWND__@@0JPAV0@@Z 10001af3 f   AccessBridgeJavaVMInstance.obj
 0001:00000b3f       ??1AccessBridgeJavaVMInstance@@QAE@XZ 10001b3f f   AccessBridgeJavaVMInstance.obj
 0001:00000b89       ?findABJavaVMInstanceFromJavaHWND@AccessBridgeJavaVMInstance@@QAEPAV1@PAUHWND__@@@Z 10001b89 f   AccessBridgeJavaVMInstance.obj
 0001:00000bc5       ?findAccessBridgeWindow@AccessBridgeJavaVMInstance@@QAEPAUHWND__@@J@Z 10001bc5 f   AccessBridgeJavaVMInstance.obj
 0001:00000c0c       ?initiateIPC@AccessBridgeJavaVMInstance@@QAEJXZ 10001c0c f   AccessBridgeJavaVMInstance.obj
 0001:00000ccb       ?sendMemoryPackage@AccessBridgeJavaVMInstance@@QAEHPADJ@Z 10001ccb f   AccessBridgeJavaVMInstance.obj
 0001:00000d83       ?sendPackage@AccessBridgeJavaVMInstance@@QAEJPADJ@Z 10001d83 f   AccessBridgeJavaVMInstance.obj
 0001:00000dd8       _snprintf                  10001dd8 f i AccessBridgeJavaVMInstance.obj
 0001:00000df2       _vsnprintf                 10001df2 f i AccessBridgeJavaVMInstance.obj
 0001:00000e24       ??0AccessBridgeMessageQueue@@QAE@XZ 10001e24 f   AccessBridgeMessageQueue.obj
 0001:00000e37       ??0AccessBridgeQueueElement@@QAE@PADH@Z 10001e37 f   AccessBridgeMessageQueue.obj
 0001:00000e89       ??0bad_alloc@std@@QAE@ABV01@@Z 10001e89 f i AccessBridgeMessageQueue.obj
 0001:00000ea1       ??0bad_alloc@std@@QAE@XZ   10001ea1 f i AccessBridgeMessageQueue.obj
 0001:00000eb9       ??0exception@std@@QAE@ABV01@@Z 10001eb9 f i AccessBridgeMessageQueue.obj
 0001:00000ee2       ??1AccessBridgeQueueElement@@QAE@XZ 10001ee2 f   AccessBridgeMessageQueue.obj
 0001:00000eec       ??1bad_alloc@std@@UAE@XZ   10001eec f i AccessBridgeMessageQueue.obj
 0001:00000eec       ??1bad_array_new_length@std@@UAE@XZ 10001eec f i MSVCRT:throw_bad_alloc.obj
 0001:00000efd       ??_Ebad_alloc@std@@UAEPAXI@Z 10001efd f i AccessBridgeMessageQueue.obj
 0001:00000efd       ??_Eexception@std@@UAEPAXI@Z 10001efd f i AccessBridgeMessageQueue.obj
 0001:00000efd       ??_Gbad_alloc@std@@UAEPAXI@Z 10001efd f i AccessBridgeMessageQueue.obj
 0001:00000efd       ??_Gexception@std@@UAEPAXI@Z 10001efd f i AccessBridgeMessageQueue.obj
 0001:00000f27       ?add@AccessBridgeMessageQueue@@QAE?AW4QueueReturns@@PAVAccessBridgeQueueElement@@@Z 10001f27 f   AccessBridgeMessageQueue.obj
 0001:00000fc3       ?getEventsWaiting@AccessBridgeMessageQueue@@QAEHXZ 10001fc3 f   AccessBridgeMessageQueue.obj
 0001:00000fc7       ?getRemoveLockSetting@AccessBridgeMessageQueue@@QAEHXZ 10001fc7 f   AccessBridgeMessageQueue.obj
 0001:00000fcb       ?remove@AccessBridgeMessageQueue@@QAE?AW4QueueReturns@@PAPAVAccessBridgeQueueElement@@@Z 10001fcb f   AccessBridgeMessageQueue.obj
 0001:00001061       ?setRemoveLock@AccessBridgeMessageQueue@@QAE?AW4QueueReturns@@H@Z 10002061 f   AccessBridgeMessageQueue.obj
 0001:00001077       ?what@exception@std@@UBEPBDXZ 10002077 f i AccessBridgeMessageQueue.obj
 0001:00001085       ?initBroadcastMessageIDs@@YAHXZ 10002085 f   AccessBridgeMessages.obj
 0001:000010b8       _Windows_run               100020b8 f   AccessBridgeWindowsEntryPoints.obj
 0001:000010c7       _activateAccessibleHyperlink 100020c7 f   AccessBridgeWindowsEntryPoints.obj
 0001:000010e6       _addAccessibleSelectionFromContext 100020e6 f   AccessBridgeWindowsEntryPoints.obj
 0001:00001102       _clearAccessibleSelectionFromContext 10002102 f   AccessBridgeWindowsEntryPoints.obj
 0001:0000111a       _doAccessibleActions       1000211a f   AccessBridgeWindowsEntryPoints.obj
 0001:0000113d       _getAccessibleActions      1000213d f   AccessBridgeWindowsEntryPoints.obj
 0001:0000115c       _getAccessibleChildFromContext 1000215c f   AccessBridgeWindowsEntryPoints.obj
 0001:0000117b       _getAccessibleContextAt    1000217b f   AccessBridgeWindowsEntryPoints.obj
 0001:000011a2       _getAccessibleContextFromHWND 100021a2 f   AccessBridgeWindowsEntryPoints.obj
 0001:000011c1       _getAccessibleContextInfo  100021c1 f   AccessBridgeWindowsEntryPoints.obj
 0001:000011e0       _getAccessibleContextWithFocus 100021e0 f   AccessBridgeWindowsEntryPoints.obj
 0001:000011ff       _getAccessibleHyperlink    100021ff f   AccessBridgeWindowsEntryPoints.obj
 0001:00001222       _getAccessibleHyperlinkCount 10002222 f   AccessBridgeWindowsEntryPoints.obj
 0001:0000123e       _getAccessibleHypertext    1000223e f   AccessBridgeWindowsEntryPoints.obj
 0001:0000125d       _getAccessibleHypertextExt 1000225d f   AccessBridgeWindowsEntryPoints.obj
 0001:00001280       _getAccessibleHypertextLinkIndex 10002280 f   AccessBridgeWindowsEntryPoints.obj
 0001:000012a0       _getAccessibleIcons        100022a0 f   AccessBridgeWindowsEntryPoints.obj
 0001:000012bf       _getAccessibleKeyBindings  100022bf f   AccessBridgeWindowsEntryPoints.obj
 0001:000012de       _getAccessibleParentFromContext 100022de f   AccessBridgeWindowsEntryPoints.obj
 0001:000012f9       _getAccessibleRelationSet  100022f9 f   AccessBridgeWindowsEntryPoints.obj
 0001:00001318       _getAccessibleSelectionCountFromContext 10002318 f   AccessBridgeWindowsEntryPoints.obj
 0001:00001334       _getAccessibleSelectionFromContext 10002334 f   AccessBridgeWindowsEntryPoints.obj
 0001:00001353       _getAccessibleTableCellInfo 10002353 f   AccessBridgeWindowsEntryPoints.obj
 0001:0000137a       _getAccessibleTableColumn  1000237a f   AccessBridgeWindowsEntryPoints.obj
 0001:0000139a       _getAccessibleTableColumnDescription 1000239a f   AccessBridgeWindowsEntryPoints.obj
 0001:000013b9       _getAccessibleTableColumnHeader 100023b9 f   AccessBridgeWindowsEntryPoints.obj
 0001:000013d8       _getAccessibleTableColumnSelectionCount 100023d8 f   AccessBridgeWindowsEntryPoints.obj
 0001:000013f4       _getAccessibleTableColumnSelections 100023f4 f   AccessBridgeWindowsEntryPoints.obj
 0001:00001417       _getAccessibleTableIndex   10002417 f   AccessBridgeWindowsEntryPoints.obj
 0001:0000143b       _getAccessibleTableInfo    1000243b f   AccessBridgeWindowsEntryPoints.obj
 0001:0000145a       _getAccessibleTableRow     1000245a f   AccessBridgeWindowsEntryPoints.obj
 0001:0000147a       _getAccessibleTableRowDescription 1000247a f   AccessBridgeWindowsEntryPoints.obj
 0001:00001499       _getAccessibleTableRowHeader 10002499 f   AccessBridgeWindowsEntryPoints.obj
 0001:000014b8       _getAccessibleTableRowSelectionCount 100024b8 f   AccessBridgeWindowsEntryPoints.obj
 0001:000014d4       _getAccessibleTableRowSelections 100024d4 f   AccessBridgeWindowsEntryPoints.obj
 0001:000014f7       _getAccessibleTextAttributes 100024f7 f   AccessBridgeWindowsEntryPoints.obj
 0001:0000151a       _getAccessibleTextInfo     1000251a f   AccessBridgeWindowsEntryPoints.obj
 0001:00001541       _getAccessibleTextItems    10002541 f   AccessBridgeWindowsEntryPoints.obj
 0001:00001564       _getAccessibleTextLineBounds 10002564 f   AccessBridgeWindowsEntryPoints.obj
 0001:0000158b       _getAccessibleTextRange    1000258b f   AccessBridgeWindowsEntryPoints.obj
 0001:000015b5       _getAccessibleTextRect     100025b5 f   AccessBridgeWindowsEntryPoints.obj
 0001:000015d8       _getAccessibleTextSelectionInfo 100025d8 f   AccessBridgeWindowsEntryPoints.obj
 0001:000015f7       _getActiveDescendent       100025f7 f   AccessBridgeWindowsEntryPoints.obj
 0001:00001612       _getCaretLocation          10002612 f   AccessBridgeWindowsEntryPoints.obj
 0001:00001635       _getCurrentAccessibleValueFromContext 10002635 f   AccessBridgeWindowsEntryPoints.obj
 0001:00001658       _getEventsWaiting          10002658 f   AccessBridgeWindowsEntryPoints.obj
 0001:00001669       _getHWNDFromAccessibleContext 10002669 f   AccessBridgeWindowsEntryPoints.obj
 0001:00001684       _getMaximumAccessibleValueFromContext 10002684 f   AccessBridgeWindowsEntryPoints.obj
 0001:000016a7       _getMinimumAccessibleValueFromContext 100026a7 f   AccessBridgeWindowsEntryPoints.obj
 0001:000016ca       _getObjectDepth            100026ca f   AccessBridgeWindowsEntryPoints.obj
 0001:000016e6       _getParentWithRole         100026e6 f   AccessBridgeWindowsEntryPoints.obj
 0001:00001705       _getParentWithRoleElseRoot 10002705 f   AccessBridgeWindowsEntryPoints.obj
 0001:00001724       _getTextAttributesInRange  10002724 f   AccessBridgeWindowsEntryPoints.obj
 0001:0000174e       _getTopLevelHWND           1000274e f   AccessBridgeWindowsEntryPoints.obj
 0001:00001786       _getTopLevelObject         10002786 f   AccessBridgeWindowsEntryPoints.obj
 0001:000017a1       _getVersionInfo            100027a1 f   AccessBridgeWindowsEntryPoints.obj
 0001:000017b9       _getVirtualAccessibleName  100027b9 f   AccessBridgeWindowsEntryPoints.obj
 0001:000017dc       _getVisibleChildren        100027dc f   AccessBridgeWindowsEntryPoints.obj
 0001:000017ff       _getVisibleChildrenCount   100027ff f   AccessBridgeWindowsEntryPoints.obj
 0001:0000181a       _isAccessibleChildSelectedFromContext 1000281a f   AccessBridgeWindowsEntryPoints.obj
 0001:00001839       _isAccessibleTableColumnSelected 10002839 f   AccessBridgeWindowsEntryPoints.obj
 0001:00001858       _isAccessibleTableRowSelected 10002858 f   AccessBridgeWindowsEntryPoints.obj
 0001:00001877       _isJavaWindow              10002877 f   AccessBridgeWindowsEntryPoints.obj
 0001:0000188e       _isSameObject              1000288e f   AccessBridgeWindowsEntryPoints.obj
 0001:000018c2       _releaseJavaObject         100028c2 f   AccessBridgeWindowsEntryPoints.obj
 0001:000018da       _removeAccessibleSelectionFromContext 100028da f   AccessBridgeWindowsEntryPoints.obj
 0001:000018f6       _requestFocus              100028f6 f   AccessBridgeWindowsEntryPoints.obj
 0001:00001911       _selectAllAccessibleSelectionFromContext 10002911 f   AccessBridgeWindowsEntryPoints.obj
 0001:00001929       _selectTextRange           10002929 f   AccessBridgeWindowsEntryPoints.obj
 0001:0000194c       _setCaretPosition          1000294c f   AccessBridgeWindowsEntryPoints.obj
 0001:0000196b       _setCaretUpdateFP          1000296b f   AccessBridgeWindowsEntryPoints.obj
 0001:0000197f       _setFocusGainedFP          1000297f f   AccessBridgeWindowsEntryPoints.obj
 0001:00001993       _setFocusLostFP            10002993 f   AccessBridgeWindowsEntryPoints.obj
 0001:000019a7       _setJavaShutdownFP         100029a7 f   AccessBridgeWindowsEntryPoints.obj
 0001:000019bb       _setMenuCanceledFP         100029bb f   AccessBridgeWindowsEntryPoints.obj
 0001:000019cf       _setMenuDeselectedFP       100029cf f   AccessBridgeWindowsEntryPoints.obj
 0001:000019e3       _setMenuSelectedFP         100029e3 f   AccessBridgeWindowsEntryPoints.obj
 0001:000019f7       _setMouseClickedFP         100029f7 f   AccessBridgeWindowsEntryPoints.obj
 0001:00001a0b       _setMouseEnteredFP         10002a0b f   AccessBridgeWindowsEntryPoints.obj
 0001:00001a1f       _setMouseExitedFP          10002a1f f   AccessBridgeWindowsEntryPoints.obj
 0001:00001a33       _setMousePressedFP         10002a33 f   AccessBridgeWindowsEntryPoints.obj
 0001:00001a47       _setMouseReleasedFP        10002a47 f   AccessBridgeWindowsEntryPoints.obj
 0001:00001a5b       _setPopupMenuCanceledFP    10002a5b f   AccessBridgeWindowsEntryPoints.obj
 0001:00001a6f       _setPopupMenuWillBecomeInvisibleFP 10002a6f f   AccessBridgeWindowsEntryPoints.obj
 0001:00001a83       _setPopupMenuWillBecomeVisibleFP 10002a83 f   AccessBridgeWindowsEntryPoints.obj
 0001:00001a97       _setPropertyActiveDescendentChangeFP 10002a97 f   AccessBridgeWindowsEntryPoints.obj
 0001:00001aab       _setPropertyCaretChangeFP  10002aab f   AccessBridgeWindowsEntryPoints.obj
 0001:00001abf       _setPropertyChangeFP       10002abf f   AccessBridgeWindowsEntryPoints.obj
 0001:00001ad3       _setPropertyChildChangeFP  10002ad3 f   AccessBridgeWindowsEntryPoints.obj
 0001:00001ae7       _setPropertyDescriptionChangeFP 10002ae7 f   AccessBridgeWindowsEntryPoints.obj
 0001:00001afb       _setPropertyNameChangeFP   10002afb f   AccessBridgeWindowsEntryPoints.obj
 0001:00001b0f       _setPropertySelectionChangeFP 10002b0f f   AccessBridgeWindowsEntryPoints.obj
 0001:00001b23       _setPropertyStateChangeFP  10002b23 f   AccessBridgeWindowsEntryPoints.obj
 0001:00001b37       _setPropertyTableModelChangeFP 10002b37 f   AccessBridgeWindowsEntryPoints.obj
 0001:00001b4b       _setPropertyTextChangeFP   10002b4b f   AccessBridgeWindowsEntryPoints.obj
 0001:00001b5f       _setPropertyValueChangeFP  10002b5f f   AccessBridgeWindowsEntryPoints.obj
 0001:00001b73       _setPropertyVisibleDataChangeFP 10002b73 f   AccessBridgeWindowsEntryPoints.obj
 0001:00001b87       _setTextContents           10002b87 f   AccessBridgeWindowsEntryPoints.obj
 0001:00001ba6       ??0WinAccessBridge@@QAE@PAUHINSTANCE__@@@Z 10002ba6 f   WinAccessBridge.obj
 0001:00001c24       ??1WinAccessBridge@@QAE@XZ 10002c24 f   WinAccessBridge.obj
 0001:00001ce1       ?JavaVMDestroyed@WinAccessBridge@@QAEXPAUHWND__@@@Z 10002ce1 f   WinAccessBridge.obj
 0001:00001d7b       ?activateAccessibleHyperlink@WinAccessBridge@@QAEHJPAV_jobject@@0@Z 10002d7b f   WinAccessBridge.obj
 0001:00001dfb       ?addAccessibilityEventNotification@WinAccessBridge@@QAEX_J@Z 10002dfb f   WinAccessBridge.obj
 0001:00001e87       ?addAccessibleSelectionFromContext@WinAccessBridge@@QAEXJPAV_jobject@@H@Z 10002e87 f   WinAccessBridge.obj
 0001:00001ee1       ?addJavaEventNotification@WinAccessBridge@@QAEX_J@Z 10002ee1 f   WinAccessBridge.obj
 0001:00001f6d       ?clearAccessibleSelectionFromContext@WinAccessBridge@@QAEXJPAV_jobject@@@Z 10002f6d f   WinAccessBridge.obj
 0001:00001fc1       ?doAccessibleActions@WinAccessBridge@@QAEHJPAV_jobject@@PAUAccessibleActionsToDoTag@@PAJ@Z 10002fc1 f   WinAccessBridge.obj
 0001:0000209d       ?getAccessibleActions@WinAccessBridge@@QAEHJPAV_jobject@@PAUAccessibleActionsTag@@@Z 1000309d f   WinAccessBridge.obj
 0001:0000216e       ?getAccessibleChildFromContext@WinAccessBridge@@QAEPAV_jobject@@JPAV2@J@Z 1000316e f   WinAccessBridge.obj
 0001:000021e8       ?getAccessibleContextAt@WinAccessBridge@@QAEHJPAV_jobject@@JJPAPAV2@@Z 100031e8 f   WinAccessBridge.obj
 0001:0000226e       ?getAccessibleContextFromHWND@WinAccessBridge@@QAEHPAUHWND__@@PAJPAPAV_jobject@@@Z 1000326e f   WinAccessBridge.obj
 0001:0000235c       ?getAccessibleContextInfo@WinAccessBridge@@QAEHJPAV_jobject@@PAUAccessibleContextInfoTag@@@Z 1000335c f   WinAccessBridge.obj
 0001:00002431       ?getAccessibleContextWithFocus@WinAccessBridge@@QAEHPAUHWND__@@PAJPAPAV_jobject@@@Z 10003431 f   WinAccessBridge.obj
 0001:000024cb       ?getAccessibleHyperlink@WinAccessBridge@@QAEHJQAV_jobject@@JPAUAccessibleHyperlinkInfoTag@@@Z 100034cb f   WinAccessBridge.obj
 0001:00002597       ?getAccessibleHyperlinkCount@WinAccessBridge@@QAEJJQAV_jobject@@@Z 10003597 f   WinAccessBridge.obj
 0001:00002634       ?getAccessibleHypertext@WinAccessBridge@@QAEHJPAV_jobject@@PAUAccessibleHypertextInfoTag@@@Z 10003634 f   WinAccessBridge.obj
 0001:00002705       ?getAccessibleHypertextExt@WinAccessBridge@@QAEHJQAV_jobject@@JPAUAccessibleHypertextInfoTag@@@Z 10003705 f   WinAccessBridge.obj
 0001:00002808       ?getAccessibleHypertextLinkIndex@WinAccessBridge@@QAEJJQAV_jobject@@J@Z 10003808 f   WinAccessBridge.obj
 0001:000028ab       ?getAccessibleIcons@WinAccessBridge@@QAEHJPAV_jobject@@PAUAccessibleIconsTag@@@Z 100038ab f   WinAccessBridge.obj
 0001:0000297c       ?getAccessibleKeyBindings@WinAccessBridge@@QAEHJPAV_jobject@@PAUAccessibleKeyBindingsTag@@@Z 1000397c f   WinAccessBridge.obj
 0001:00002a5a       ?getAccessibleParentFromContext@WinAccessBridge@@QAEPAV_jobject@@JPAV2@@Z 10003a5a f   WinAccessBridge.obj
 0001:00002acd       ?getAccessibleRelationSet@WinAccessBridge@@QAEHJPAV_jobject@@PAUAccessibleRelationSetInfoTag@@@Z 10003acd f   WinAccessBridge.obj
 0001:00002b9c       ?getAccessibleSelectionCountFromContext@WinAccessBridge@@QAEHJPAV_jobject@@@Z 10003b9c f   WinAccessBridge.obj
 0001:00002bfd       ?getAccessibleSelectionFromContext@WinAccessBridge@@QAEPAV_jobject@@JPAV2@H@Z 10003bfd f   WinAccessBridge.obj
 0001:00002c63       ?getAccessibleTableCellInfo@WinAccessBridge@@QAEHJPAV_jobject@@JJPAUAccessibleTableCellInfoTag@@@Z 10003c63 f   WinAccessBridge.obj
 0001:00002d2f       ?getAccessibleTableColumn@WinAccessBridge@@QAEJJPAV_jobject@@J@Z 10003d2f f   WinAccessBridge.obj
 0001:00002dcb       ?getAccessibleTableColumnDescription@WinAccessBridge@@QAEPAV_jobject@@JPAV2@J@Z 10003dcb f   WinAccessBridge.obj
 0001:00002e67       ?getAccessibleTableColumnHeader@WinAccessBridge@@QAEHJPAV_jobject@@PAUAccessibleTableInfoTag@@@Z 10003e67 f   WinAccessBridge.obj
 0001:00002f0c       ?getAccessibleTableColumnSelectionCount@WinAccessBridge@@QAEJJPAV_jobject@@@Z 10003f0c f   WinAccessBridge.obj
 0001:00002f95       ?getAccessibleTableColumnSelections@WinAccessBridge@@QAEHJPAV_jobject@@JPAJ@Z 10003f95 f   WinAccessBridge.obj
 0001:0000306c       ?getAccessibleTableIndex@WinAccessBridge@@QAEJJPAV_jobject@@JJ@Z 1000406c f   WinAccessBridge.obj
 0001:00003114       ?getAccessibleTableInfo@WinAccessBridge@@QAEHJPAV_jobject@@PAUAccessibleTableInfoTag@@@Z 10004114 f   WinAccessBridge.obj
 0001:000031c2       ?getAccessibleTableRow@WinAccessBridge@@QAEJJPAV_jobject@@J@Z 100041c2 f   WinAccessBridge.obj
 0001:0000325e       ?getAccessibleTableRowDescription@WinAccessBridge@@QAEPAV_jobject@@JPAV2@J@Z 1000425e f   WinAccessBridge.obj
 0001:000032fa       ?getAccessibleTableRowHeader@WinAccessBridge@@QAEHJPAV_jobject@@PAUAccessibleTableInfoTag@@@Z 100042fa f   WinAccessBridge.obj
 0001:0000339f       ?getAccessibleTableRowSelectionCount@WinAccessBridge@@QAEJJPAV_jobject@@@Z 1000439f f   WinAccessBridge.obj
 0001:00003428       ?getAccessibleTableRowSelections@WinAccessBridge@@QAEHJPAV_jobject@@JPAJ@Z 10004428 f   WinAccessBridge.obj
 0001:000034f4       ?getAccessibleTextAttributes@WinAccessBridge@@QAEHJPAV_jobject@@JPAUAccessibleTextAttributesInfoTag@@@Z 100044f4 f   WinAccessBridge.obj
 0001:0000359e       ?getAccessibleTextInfo@WinAccessBridge@@QAEHJPAV_jobject@@PAUAccessibleTextInfoTag@@JJ@Z 1000459e f   WinAccessBridge.obj
 0001:0000364f       ?getAccessibleTextItems@WinAccessBridge@@QAEHJPAV_jobject@@PAUAccessibleTextItemsInfoTag@@J@Z 1000464f f   WinAccessBridge.obj
 0001:0000371a       ?getAccessibleTextLineBounds@WinAccessBridge@@QAEHJPAV_jobject@@JPAJ1@Z 1000471a f   WinAccessBridge.obj
 0001:000037b3       ?getAccessibleTextRange@WinAccessBridge@@QAEHJPAV_jobject@@JJPAGF@Z 100047b3 f   WinAccessBridge.obj
 0001:0000386b       ?getAccessibleTextRect@WinAccessBridge@@QAEHJPAV_jobject@@PAUAccessibleTextRectInfoTag@@J@Z 1000486b f   WinAccessBridge.obj
 0001:000038fa       ?getAccessibleTextSelectionInfo@WinAccessBridge@@QAEHJPAV_jobject@@PAUAccessibleTextSelectionInfoTag@@@Z 100048fa f   WinAccessBridge.obj
 0001:0000399a       ?getActiveDescendent@WinAccessBridge@@QAEPAV_jobject@@JQAV2@@Z 1000499a f   WinAccessBridge.obj
 0001:00003a0d       ?getCaretLocation@WinAccessBridge@@QAEHJPAV_jobject@@PAUAccessibleTextRectInfoTag@@J@Z 10004a0d f   WinAccessBridge.obj
 0001:00003a9c       ?getCurrentAccessibleValueFromContext@WinAccessBridge@@QAEHJPAV_jobject@@PAGF@Z 10004a9c f   WinAccessBridge.obj
 0001:00003b29       ?getEventsWaiting@WinAccessBridge@@QAEHXZ 10004b29 f   WinAccessBridge.obj
 0001:00003b37       ?getHWNDFromAccessibleContext@WinAccessBridge@@QAEPAUHWND__@@JPAV_jobject@@@Z 10004b37 f   WinAccessBridge.obj
 0001:00003bb2       ?getMaximumAccessibleValueFromContext@WinAccessBridge@@QAEHJPAV_jobject@@PAGF@Z 10004bb2 f   WinAccessBridge.obj
 0001:00003c3f       ?getMinimumAccessibleValueFromContext@WinAccessBridge@@QAEHJPAV_jobject@@PAGF@Z 10004c3f f   WinAccessBridge.obj
 0001:00003ccc       ?getObjectDepth@WinAccessBridge@@QAEHJQAV_jobject@@@Z 10004ccc f   WinAccessBridge.obj
 0001:00003d40       ?getParentWithRole@WinAccessBridge@@QAEPAV_jobject@@JQAV2@PBG@Z 10004d40 f   WinAccessBridge.obj
 0001:00003e0c       ?getParentWithRoleElseRoot@WinAccessBridge@@QAEPAV_jobject@@JQAV2@PBG@Z 10004e0c f   WinAccessBridge.obj
 0001:00003ea8       ?getTextAttributesInRange@WinAccessBridge@@QAEHJPAV_jobject@@HHPAUAccessibleTextAttributesInfoTag@@PAF@Z 10004ea8 f   WinAccessBridge.obj
 0001:00003fa1       ?getTopLevelObject@WinAccessBridge@@QAEPAV_jobject@@JQAV2@@Z 10004fa1 f   WinAccessBridge.obj
 0001:00004014       ?getVersionInfo@WinAccessBridge@@QAEHJPAUAccessBridgeVersionInfoTag@@@Z 10005014 f   WinAccessBridge.obj
 0001:000040c8       ?getVirtualAccessibleName@WinAccessBridge@@QAEHJPAV_jobject@@PAGH@Z 100050c8 f   WinAccessBridge.obj
 0001:00004195       ?getVisibleChildren@WinAccessBridge@@QAEHJPAV_jobject@@HPAUVisibleChildenInfoTag@@@Z 10005195 f   WinAccessBridge.obj
 0001:0000423d       ?getVisibleChildrenCount@WinAccessBridge@@QAEHJPAV_jobject@@@Z 1000523d f   WinAccessBridge.obj
 0001:000042b1       ?initWindow@WinAccessBridge@@QAEHXZ 100052b1 f   WinAccessBridge.obj
 0001:000042f6       ?isAccessibleChildSelectedFromContext@WinAccessBridge@@QAEHJPAV_jobject@@H@Z 100052f6 f   WinAccessBridge.obj
 0001:00004361       ?isAccessibleTableColumnSelected@WinAccessBridge@@QAEHJPAV_jobject@@J@Z 10005361 f   WinAccessBridge.obj
 0001:000043f1       ?isAccessibleTableRowSelected@WinAccessBridge@@QAEHJPAV_jobject@@J@Z 100053f1 f   WinAccessBridge.obj
 0001:00004481       ?isJavaWindow@WinAccessBridge@@QAEHPAUHWND__@@@Z 10005481 f   WinAccessBridge.obj
 0001:0000451d       ?isSameObject@WinAccessBridge@@QAEHJPAV_jobject@@0@Z 1000551d f   WinAccessBridge.obj
 0001:000045b5       ?preProcessPackage@WinAccessBridge@@QAEXPADJ@Z 100055b5 f   WinAccessBridge.obj
 0001:00004694       ?processPackage@WinAccessBridge@@QAEXPADJ@Z 10005694 f   WinAccessBridge.obj
 0001:00004d77       ?queuePackage@WinAccessBridge@@QAEHPADJ@Z 10005d77 f   WinAccessBridge.obj
 0001:00004dcf       ?receiveAQueuedPackage@WinAccessBridge@@QAEHXZ 10005dcf f   WinAccessBridge.obj
 0001:00004ec7       ?releaseJavaObject@WinAccessBridge@@QAEXJPAV_jobject@@@Z 10005ec7 f   WinAccessBridge.obj
 0001:00004f2e       ?removeAccessibilityEventNotification@WinAccessBridge@@QAEX_J@Z 10005f2e f   WinAccessBridge.obj
 0001:00004fba       ?removeAccessibleSelectionFromContext@WinAccessBridge@@QAEXJPAV_jobject@@H@Z 10005fba f   WinAccessBridge.obj
 0001:00005014       ?removeJavaEventNotification@WinAccessBridge@@QAEX_J@Z 10006014 f   WinAccessBridge.obj
 0001:000050a0       ?rendezvousWithNewJavaDLL@WinAccessBridge@@QAEJPAUHWND__@@J@Z 100060a0 f   WinAccessBridge.obj
 0001:00005160       ?requestFocus@WinAccessBridge@@QAEHJPAV_jobject@@@Z 10006160 f   WinAccessBridge.obj
 0001:000051d1       ?selectAllAccessibleSelectionFromContext@WinAccessBridge@@QAEXJPAV_jobject@@@Z 100061d1 f   WinAccessBridge.obj
 0001:00005225       ?selectTextRange@WinAccessBridge@@QAEHJPAV_jobject@@HH@Z 10006225 f   WinAccessBridge.obj
 0001:000052a4       ?sendMemoryPackage@WinAccessBridge@@QAEHPADJPAUHWND__@@@Z 100062a4 f   WinAccessBridge.obj
 0001:000052f2       ?sendPackage@WinAccessBridge@@QAEXPADJPAUHWND__@@@Z 100062f2 f   WinAccessBridge.obj
 0001:0000531e       ?setCaretPosition@WinAccessBridge@@QAEHJPAV_jobject@@H@Z 1000631e f   WinAccessBridge.obj
 0001:00005395       ?setCaretUpdateFP@WinAccessBridge@@QAEXP6AXJPAV_jobject@@0@Z@Z 10006395 f   WinAccessBridge.obj
 0001:000053a5       ?setFocusGainedFP@WinAccessBridge@@QAEXP6AXJPAV_jobject@@0@Z@Z 100063a5 f   WinAccessBridge.obj
 0001:000053b5       ?setFocusLostFP@WinAccessBridge@@QAEXP6AXJPAV_jobject@@0@Z@Z 100063b5 f   WinAccessBridge.obj
 0001:000053c5       ?setJavaShutdownFP@WinAccessBridge@@QAEXP6AXJ@Z@Z 100063c5 f   WinAccessBridge.obj
 0001:000053d5       ?setMenuCanceledFP@WinAccessBridge@@QAEXP6AXJPAV_jobject@@0@Z@Z 100063d5 f   WinAccessBridge.obj
 0001:000053e5       ?setMenuDeselectedFP@WinAccessBridge@@QAEXP6AXJPAV_jobject@@0@Z@Z 100063e5 f   WinAccessBridge.obj
 0001:000053f5       ?setMenuSelectedFP@WinAccessBridge@@QAEXP6AXJPAV_jobject@@0@Z@Z 100063f5 f   WinAccessBridge.obj
 0001:00005405       ?setMouseClickedFP@WinAccessBridge@@QAEXP6AXJPAV_jobject@@0@Z@Z 10006405 f   WinAccessBridge.obj
 0001:00005415       ?setMouseEnteredFP@WinAccessBridge@@QAEXP6AXJPAV_jobject@@0@Z@Z 10006415 f   WinAccessBridge.obj
 0001:00005425       ?setMouseExitedFP@WinAccessBridge@@QAEXP6AXJPAV_jobject@@0@Z@Z 10006425 f   WinAccessBridge.obj
 0001:00005435       ?setMousePressedFP@WinAccessBridge@@QAEXP6AXJPAV_jobject@@0@Z@Z 10006435 f   WinAccessBridge.obj
 0001:00005445       ?setMouseReleasedFP@WinAccessBridge@@QAEXP6AXJPAV_jobject@@0@Z@Z 10006445 f   WinAccessBridge.obj
 0001:00005455       ?setPopupMenuCanceledFP@WinAccessBridge@@QAEXP6AXJPAV_jobject@@0@Z@Z 10006455 f   WinAccessBridge.obj
 0001:00005465       ?setPopupMenuWillBecomeInvisibleFP@WinAccessBridge@@QAEXP6AXJPAV_jobject@@0@Z@Z 10006465 f   WinAccessBridge.obj
 0001:00005475       ?setPopupMenuWillBecomeVisibleFP@WinAccessBridge@@QAEXP6AXJPAV_jobject@@0@Z@Z 10006475 f   WinAccessBridge.obj
 0001:00005485       ?setPropertyActiveDescendentChangeFP@WinAccessBridge@@QAEXP6AXJPAV_jobject@@000@Z@Z 10006485 f   WinAccessBridge.obj
 0001:00005495       ?setPropertyCaretChangeFP@WinAccessBridge@@QAEXP6AXJPAV_jobject@@0HH@Z@Z 10006495 f   WinAccessBridge.obj
 0001:000054a5       ?setPropertyChangeFP@WinAccessBridge@@QAEXP6AXJPAV_jobject@@0PAG11@Z@Z 100064a5 f   WinAccessBridge.obj
 0001:000054b5       ?setPropertyChildChangeFP@WinAccessBridge@@QAEXP6AXJPAV_jobject@@000@Z@Z 100064b5 f   WinAccessBridge.obj
 0001:000054c5       ?setPropertyDescriptionChangeFP@WinAccessBridge@@QAEXP6AXJPAV_jobject@@0PAG1@Z@Z 100064c5 f   WinAccessBridge.obj
 0001:000054d5       ?setPropertyNameChangeFP@WinAccessBridge@@QAEXP6AXJPAV_jobject@@0PAG1@Z@Z 100064d5 f   WinAccessBridge.obj
 0001:000054e5       ?setPropertySelectionChangeFP@WinAccessBridge@@QAEXP6AXJPAV_jobject@@0@Z@Z 100064e5 f   WinAccessBridge.obj
 0001:000054f5       ?setPropertyStateChangeFP@WinAccessBridge@@QAEXP6AXJPAV_jobject@@0PAG1@Z@Z 100064f5 f   WinAccessBridge.obj
 0001:00005505       ?setPropertyTableModelChangeFP@WinAccessBridge@@QAEXP6AXJPAV_jobject@@0PAG1@Z@Z 10006505 f   WinAccessBridge.obj
 0001:00005515       ?setPropertyTextChangeFP@WinAccessBridge@@QAEXP6AXJPAV_jobject@@0@Z@Z 10006515 f   WinAccessBridge.obj
 0001:00005525       ?setPropertyValueChangeFP@WinAccessBridge@@QAEXP6AXJPAV_jobject@@0PAG1@Z@Z 10006525 f   WinAccessBridge.obj
 0001:00005535       ?setPropertyVisibleDataChangeFP@WinAccessBridge@@QAEXP6AXJPAV_jobject@@0@Z@Z 10006535 f   WinAccessBridge.obj
 0001:00005545       ?setTextContents@WinAccessBridge@@QAEHJQAV_jobject@@PBG@Z 10006545 f   WinAccessBridge.obj
 0001:000055f5       _AccessBridgeDialogProc@16 100065f5 f   WinAccessBridge.obj
 0001:00005703       _DllMain@12                10006703 f   WinAccessBridge.obj
 0001:00005780       ??_U@YAPAXI@Z              10006780 f   MSVCRT:new_array.obj
 0001:00005789       ??_V@YAXPAX@Z              10006789 f   MSVCRT:delete_array.obj
 0001:00005790       __aulldiv                  10006790 f   MSVCRT:ulldiv.obj
 0001:000057f8       @__security_check_cookie@4 100067f8 f   MSVCRT:secchk.obj
 0001:00005806       ??3@YAXPAXI@Z              10006806 f   MSVCRT:delete_scalar_size.obj
 0001:00005814       ??_Etype_info@@UAEPAXI@Z   10006814 f i MSVCRT:std_type_info_static.obj
 0001:00005814       ??_Gtype_info@@UAEPAXI@Z   10006814 f i MSVCRT:std_type_info_static.obj
 0001:00005837       ??2@YAPAXI@Z               10006837 f   MSVCRT:new_scalar.obj
 0001:00005870       __alloca_probe             10006870 f   MSVCRT:chkstk.obj
 0001:00005870       __chkstk                   10006870 f   MSVCRT:chkstk.obj
 0001:00005bdb       __DllMainCRTStartup@12     10006bdb f   MSVCRT:dll_dllmain.obj
 0001:00005bfe       ??3@YAXPAX@Z               10006bfe f   MSVCRT:delete_scalar.obj
 0001:00005c03       ___raise_securityfailure   10006c03 f   MSVCRT:gs_report.obj
 0001:00005c2b       ___report_gsfailure        10006c2b f   MSVCRT:gs_report.obj
 0001:00005d25       ??0bad_array_new_length@std@@QAE@ABV01@@Z 10006d25 f i MSVCRT:throw_bad_alloc.obj
 0001:00005d40       ??0bad_array_new_length@std@@QAE@XZ 10006d40 f i MSVCRT:throw_bad_alloc.obj
 0001:00005d58       ??_Ebad_array_new_length@std@@UAEPAXI@Z 10006d58 f i MSVCRT:throw_bad_alloc.obj
 0001:00005d58       ??_Gbad_array_new_length@std@@UAEPAXI@Z 10006d58 f i MSVCRT:throw_bad_alloc.obj
 0001:00005d85       ?__scrt_throw_std_bad_alloc@@YAXXZ 10006d85 f   MSVCRT:throw_bad_alloc.obj
 0001:00005da2       ?__scrt_throw_std_bad_array_new_length@@YAXXZ 10006da2 f   MSVCRT:throw_bad_alloc.obj
 0001:00005e0c       ___security_init_cookie    10006e0c f   MSVCRT:gs_support.obj
 0001:00005e57       ?__scrt_initialize_type_info@@YAXXZ 10006e57 f   MSVCRT:tncleanup.obj
 0001:00005e63       ?__scrt_uninitialize_type_info@@YAXXZ 10006e63 f   MSVCRT:tncleanup.obj
 0001:00005e6f       ___local_stdio_scanf_options 10006e6f f i MSVCRT:default_local_stdio_options.obj
 0001:00005e75       ___scrt_initialize_default_local_stdio_options 10006e75 f   MSVCRT:default_local_stdio_options.obj
 0001:00005ed6       ___scrt_acquire_startup_lock 10006ed6 f   MSVCRT:utility.obj
 0001:00005f08       ___scrt_dllmain_after_initialize_c 10006f08 f   MSVCRT:utility.obj
 0001:00005f33       ___scrt_dllmain_before_initialize_c 10006f33 f   MSVCRT:utility.obj
 0001:00005f41       ___scrt_dllmain_crt_thread_attach 10006f41 f   MSVCRT:utility.obj
 0001:00005f60       ___scrt_dllmain_crt_thread_detach 10006f60 f   MSVCRT:utility.obj
 0001:00005f6d       ___scrt_dllmain_exception_filter 10006f6d f   MSVCRT:utility.obj
 0001:00005fa1       ___scrt_dllmain_uninitialize_c 10006fa1 f   MSVCRT:utility.obj
 0001:00005fc4       ___scrt_dllmain_uninitialize_critical 10006fc4 f   MSVCRT:utility.obj
 0001:00005fd1       ___scrt_initialize_crt     10006fd1 f   MSVCRT:utility.obj
 0001:0000600a       ___scrt_initialize_onexit_tables 1000700a f   MSVCRT:utility.obj
 0001:00006091       ___scrt_is_nonwritable_in_current_image 10007091 f   MSVCRT:utility.obj
 0001:00006125       ___scrt_release_startup_lock 10007125 f   MSVCRT:utility.obj
 0001:00006142       ___scrt_uninitialize_crt   10007142 f   MSVCRT:utility.obj
 0001:0000616a       ___scrt_get_dyn_tls_init_callback 1000716a f   MSVCRT:dyn_tls_init.obj
 0001:00006170       ___scrt_fastfail           10007170 f   MSVCRT:utility_desktop.obj
 0001:0000628b       __crt_debugger_hook        1000728b f   MSVCRT:utility_desktop.obj
 0001:00006293       __RTC_Initialize           10007293 f   MSVCRT:initsect.obj
 0001:000062bf       __RTC_Terminate            100072bf f   MSVCRT:initsect.obj
 0001:000062f0       __SEH_prolog4              100072f0 f   MSVCRT:sehprolg4.obj
 0001:00006335       __except_handler4          10007335 f   MSVCRT:chandler4gs.obj
 0001:00006364       ___isa_available_init      10007364 f   MSVCRT:cpu_disp.obj
 0001:00006538       __get_startup_argv_mode    10007538 f   MSVCRT:argv_mode.obj
 0001:0000653c       ___scrt_is_ucrt_dll_in_use 1000753c f   MSVCRT:ucrt_detection.obj
 0001:00006548       _memcpy                    10007548 f   vcruntime:VCRUNTIME140.dll
 0001:0000654e       _memset                    1000754e f   vcruntime:VCRUNTIME140.dll
 0001:00006554       ___std_exception_copy      10007554 f   vcruntime:VCRUNTIME140.dll
 0001:0000655a       ___std_exception_destroy   1000755a f   vcruntime:VCRUNTIME140.dll
 0001:00006560       __CxxThrowException@8      10007560 f   vcruntime:VCRUNTIME140.dll
 0001:00006566       ___std_type_info_destroy_list 10007566 f   vcruntime:VCRUNTIME140.dll
 0001:0000656c       __except_handler4_common   1000756c f   vcruntime:VCRUNTIME140.dll
 0001:00006572       _strlen                    10007572 f   ucrt:api-ms-win-crt-string-l1-1-0.dll
 0001:00006578       _strcmp                    10007578 f   ucrt:api-ms-win-crt-string-l1-1-0.dll
 0001:0000657e       _strcpy                    1000757e f   ucrt:api-ms-win-crt-string-l1-1-0.dll
 0001:00006584       _free                      10007584 f   ucrt:api-ms-win-crt-heap-l1-1-0.dll
 0001:0000658a       _malloc                    1000758a f   ucrt:api-ms-win-crt-heap-l1-1-0.dll
 0001:00006590       __callnewh                 10007590 f   ucrt:api-ms-win-crt-heap-l1-1-0.dll
 0001:00006596       __initterm                 10007596 f   ucrt:api-ms-win-crt-runtime-l1-1-0.dll
 0001:0000659c       __initterm_e               1000759c f   ucrt:api-ms-win-crt-runtime-l1-1-0.dll
 0001:000065a2       __seh_filter_dll           100075a2 f   ucrt:api-ms-win-crt-runtime-l1-1-0.dll
 0001:000065a8       __configure_narrow_argv    100075a8 f   ucrt:api-ms-win-crt-runtime-l1-1-0.dll
 0001:000065ae       __initialize_narrow_environment 100075ae f   ucrt:api-ms-win-crt-runtime-l1-1-0.dll
 0001:000065b4       __initialize_onexit_table  100075b4 f   ucrt:api-ms-win-crt-runtime-l1-1-0.dll
 0001:000065ba       __execute_onexit_table     100075ba f   ucrt:api-ms-win-crt-runtime-l1-1-0.dll
 0001:000065c0       __cexit                    100075c0 f   ucrt:api-ms-win-crt-runtime-l1-1-0.dll
 0001:000065c6       ___acrt_initialize         100075c6 f   MSVCRT:ucrt_stubs.obj
 0001:000065c6       ___acrt_thread_attach      100075c6 f   MSVCRT:ucrt_stubs.obj
 0001:000065c6       ___acrt_thread_detach      100075c6 f   MSVCRT:ucrt_stubs.obj
 0001:000065c6       ___acrt_uninitialize       100075c6 f   MSVCRT:ucrt_stubs.obj
 0001:000065c6       ___acrt_uninitialize_critical 100075c6 f   MSVCRT:ucrt_stubs.obj
 0001:000065c6       ___scrt_stub_for_acrt_initialize 100075c6 f   MSVCRT:ucrt_stubs.obj
 0001:000065c6       ___scrt_stub_for_acrt_thread_attach 100075c6 f   MSVCRT:ucrt_stubs.obj
 0001:000065c6       ___scrt_stub_for_acrt_thread_detach 100075c6 f   MSVCRT:ucrt_stubs.obj
 0001:000065c6       ___scrt_stub_for_acrt_uninitialize 100075c6 f   MSVCRT:ucrt_stubs.obj
 0001:000065c6       ___scrt_stub_for_acrt_uninitialize_critical 100075c6 f   MSVCRT:ucrt_stubs.obj
 0001:000065c6       ___vcrt_initialize         100075c6 f   MSVCRT:ucrt_stubs.obj
 0001:000065c6       ___vcrt_thread_attach      100075c6 f   MSVCRT:ucrt_stubs.obj
 0001:000065c6       ___vcrt_thread_detach      100075c6 f   MSVCRT:ucrt_stubs.obj
 0001:000065c6       ___vcrt_uninitialize       100075c6 f   MSVCRT:ucrt_stubs.obj
 0001:000065c6       ___vcrt_uninitialize_critical 100075c6 f   MSVCRT:ucrt_stubs.obj
 0001:000065c9       ___scrt_stub_for_is_c_termination_complete 100075c9 f   MSVCRT:ucrt_stubs.obj
 0001:000065c9       __is_c_termination_complete 100075c9 f   MSVCRT:ucrt_stubs.obj
 0001:000065cc       __filter_x86_sse2_floating_point_exception 100075cc f   MSVCRT:x86_exception_filter.obj
 0001:000065cc       __filter_x86_sse2_floating_point_exception_default 100075cc f   MSVCRT:x86_exception_filter.obj
 0002:00000000       __imp__GetLastError@0      10008000     kernel32:KERNEL32.dll
 0002:00000004       __imp__GetSystemTimeAsFileTime@4 10008004     kernel32:KERNEL32.dll
 0002:00000008       __imp__CloseHandle@4       10008008     kernel32:KERNEL32.dll
 0002:0000000c       __imp__EnterCriticalSection@4 1000800c     kernel32:KERNEL32.dll
 0002:00000010       __imp__LeaveCriticalSection@4 10008010     kernel32:KERNEL32.dll
 0002:00000014       __imp__MapViewOfFile@20    10008014     kernel32:KERNEL32.dll
 0002:00000018       __imp__UnmapViewOfFile@4   10008018     kernel32:KERNEL32.dll
 0002:0000001c       __imp__CreateFileMappingA@24 1000801c     kernel32:KERNEL32.dll
 0002:00000020       __imp__InitializeCriticalSection@4 10008020     kernel32:KERNEL32.dll
 0002:00000024       __imp__IsDebuggerPresent@0 10008024     kernel32:KERNEL32.dll
 0002:00000028       __imp__InitializeSListHead@4 10008028     kernel32:KERNEL32.dll
 0002:0000002c       __imp__GetCurrentThreadId@0 1000802c     kernel32:KERNEL32.dll
 0002:00000030       __imp__GetCurrentProcessId@0 10008030     kernel32:KERNEL32.dll
 0002:00000034       __imp__QueryPerformanceCounter@4 10008034     kernel32:KERNEL32.dll
 0002:00000038       __imp__IsProcessorFeaturePresent@4 10008038     kernel32:KERNEL32.dll
 0002:0000003c       __imp__TerminateProcess@8  1000803c     kernel32:KERNEL32.dll
 0002:00000040       __imp__GetCurrentProcess@0 10008040     kernel32:KERNEL32.dll
 0002:00000044       __imp__SetUnhandledExceptionFilter@4 10008044     kernel32:KERNEL32.dll
 0002:00000048       __imp__UnhandledExceptionFilter@4 10008048     kernel32:KERNEL32.dll
 0002:0000004c       \177KERNEL32_NULL_THUNK_DATA 1000804c     kernel32:KERNEL32.dll
 0002:00000050       __imp__ShowWindow@8        10008050     user32:USER32.dll
 0002:00000054       __imp__DestroyWindow@4     10008054     user32:USER32.dll
 0002:00000058       __imp__PostMessageA@16     10008058     user32:USER32.dll
 0002:0000005c       __imp__SendMessageA@16     1000805c     user32:USER32.dll
 0002:00000060       __imp__GetParent@4         10008060     user32:USER32.dll
 0002:00000064       __imp__GetWindowLongA@8    10008064     user32:USER32.dll
 0002:00000068       __imp__IsWindow@4          10008068     user32:USER32.dll
 0002:0000006c       __imp__RegisterWindowMessageA@4 1000806c     user32:USER32.dll
 0002:00000070       __imp__SendMessageTimeoutA@28 10008070     user32:USER32.dll
 0002:00000074       __imp__CreateDialogParamA@20 10008074     user32:USER32.dll
 0002:00000078       \177USER32_NULL_THUNK_DATA 10008078     user32:USER32.dll
 0002:0000007c       __imp___except_handler4_common 1000807c     vcruntime:VCRUNTIME140.dll
 0002:00000080       __imp___CxxThrowException@8 10008080     vcruntime:VCRUNTIME140.dll
 0002:00000084       __imp____std_exception_destroy 10008084     vcruntime:VCRUNTIME140.dll
 0002:00000088       __imp____std_exception_copy 10008088     vcruntime:VCRUNTIME140.dll
 0002:0000008c       __imp____std_type_info_destroy_list 1000808c     vcruntime:VCRUNTIME140.dll
 0002:00000090       __imp__memset              10008090     vcruntime:VCRUNTIME140.dll
 0002:00000094       __imp__memcpy              10008094     vcruntime:VCRUNTIME140.dll
 0002:00000098       \177VCRUNTIME140_NULL_THUNK_DATA 10008098     vcruntime:VCRUNTIME140.dll
 0002:0000009c       __imp__getenv              1000809c     ucrt:api-ms-win-crt-environment-l1-1-0.dll
 0002:000000a0       \177api-ms-win-crt-environment-l1-1-0_NULL_THUNK_DATA 100080a0     ucrt:api-ms-win-crt-environment-l1-1-0.dll
 0002:000000a4       __imp__free                100080a4     ucrt:api-ms-win-crt-heap-l1-1-0.dll
 0002:000000a8       __imp___callnewh           100080a8     ucrt:api-ms-win-crt-heap-l1-1-0.dll
 0002:000000ac       __imp__malloc              100080ac     ucrt:api-ms-win-crt-heap-l1-1-0.dll
 0002:000000b0       \177api-ms-win-crt-heap-l1-1-0_NULL_THUNK_DATA 100080b0     ucrt:api-ms-win-crt-heap-l1-1-0.dll
 0002:000000b4       __imp___seh_filter_dll     100080b4     ucrt:api-ms-win-crt-runtime-l1-1-0.dll
 0002:000000b8       __imp___configure_narrow_argv 100080b8     ucrt:api-ms-win-crt-runtime-l1-1-0.dll
 0002:000000bc       __imp___initialize_narrow_environment 100080bc     ucrt:api-ms-win-crt-runtime-l1-1-0.dll
 0002:000000c0       __imp___initterm           100080c0     ucrt:api-ms-win-crt-runtime-l1-1-0.dll
 0002:000000c4       __imp___execute_onexit_table 100080c4     ucrt:api-ms-win-crt-runtime-l1-1-0.dll
 0002:000000c8       __imp___cexit              100080c8     ucrt:api-ms-win-crt-runtime-l1-1-0.dll
 0002:000000cc       __imp___initterm_e         100080cc     ucrt:api-ms-win-crt-runtime-l1-1-0.dll
 0002:000000d0       __imp___initialize_onexit_table 100080d0     ucrt:api-ms-win-crt-runtime-l1-1-0.dll
 0002:000000d4       \177api-ms-win-crt-runtime-l1-1-0_NULL_THUNK_DATA 100080d4     ucrt:api-ms-win-crt-runtime-l1-1-0.dll
 0002:000000d8       __imp____acrt_iob_func     100080d8     ucrt:api-ms-win-crt-stdio-l1-1-0.dll
 0002:000000dc       __imp____stdio_common_vfprintf 100080dc     ucrt:api-ms-win-crt-stdio-l1-1-0.dll
 0002:000000e0       __imp__fclose              100080e0     ucrt:api-ms-win-crt-stdio-l1-1-0.dll
 0002:000000e4       __imp____stdio_common_vsprintf 100080e4     ucrt:api-ms-win-crt-stdio-l1-1-0.dll
 0002:000000e8       __imp__fopen               100080e8     ucrt:api-ms-win-crt-stdio-l1-1-0.dll
 0002:000000ec       \177api-ms-win-crt-stdio-l1-1-0_NULL_THUNK_DATA 100080ec     ucrt:api-ms-win-crt-stdio-l1-1-0.dll
 0002:000000f0       __imp__wcsncpy             100080f0     ucrt:api-ms-win-crt-string-l1-1-0.dll
 0002:000000f4       __imp__strcpy              100080f4     ucrt:api-ms-win-crt-string-l1-1-0.dll
 0002:000000f8       __imp__strncpy             100080f8     ucrt:api-ms-win-crt-string-l1-1-0.dll
 0002:000000fc       __imp__strlen              100080fc     ucrt:api-ms-win-crt-string-l1-1-0.dll
 0002:00000100       __imp__strcmp              10008100     ucrt:api-ms-win-crt-string-l1-1-0.dll
 0002:00000104       \177api-ms-win-crt-string-l1-1-0_NULL_THUNK_DATA 10008104     ucrt:api-ms-win-crt-string-l1-1-0.dll
 0002:00000108       ___guard_check_icall_fptr  10008108     MSVCRT:guard_support.obj
 0002:0000010c       ___castguard_check_failure_os_handled_fptr 1000810c     MSVCRT:guard_support.obj
 0002:00000110       ___xc_a                    10008110     MSVCRT:initializers.obj
 0002:00000114       ___xc_z                    10008114     MSVCRT:initializers.obj
 0002:00000118       ___xi_a                    10008118     MSVCRT:initializers.obj
 0002:0000011c       ___xi_z                    1000811c     MSVCRT:initializers.obj
 0002:00000120       ___xp_a                    10008120     MSVCRT:initializers.obj
 0002:00000124       ___xp_z                    10008124     MSVCRT:initializers.obj
 0002:00000128       ___xt_a                    10008128     MSVCRT:initializers.obj
 0002:0000012c       ___xt_z                    1000812c     MSVCRT:initializers.obj
 0002:00000130       ??_C@_0BJ@FKCDJFDK@JAVA_ACCESSBRIDGE_LOGDIR@ 10008130     AccessBridgeDebug.obj
 0002:0000014c       ??_C@_04FPOLKAEB@?4log@    1000814c     AccessBridgeDebug.obj
 0002:00000154       ??_C@_01NOFIACDB@w@        10008154     AccessBridgeDebug.obj
 0002:00000158       ??_C@_04EINJHBMM@?6?$CFs?6@ 10008158     AccessBridgeDebug.obj
 0002:00000160       ??_C@_0BH@PPBGFLKL@Could?5not?5open?5file?5?$CFs@ 10008160     AccessBridgeDebug.obj
 0002:00000178       ??_C@_07IBOBEFLP@?$FL?$CFllu?$FN?5@ 10008178     AccessBridgeDebug.obj
 0002:00000180       ??_C@_02PCIJFNDE@?$AN?6@   10008180     AccessBridgeDebug.obj
 0002:00000184       ??_C@_0BH@BLGOOJIK@AccessBridge?9?$CFp?9?$CFp?4mmf@ 10008184     AccessBridgeJavaVMInstance.obj
 0002:0000019c       ??_C@_03DJNNCAJF@OK?$DP@   1000819c     AccessBridgeJavaVMInstance.obj
 0002:000001a0       ??_C@_03ONJMBPEK@OK?$CB@   100081a0     AccessBridgeJavaVMInstance.obj
 0002:000001a4       ??_C@_0CP@JIGBIHFH@?$FLINFO?$FN?3?5In?5AccessBridgeVMInstan@ 100081a4     AccessBridgeJavaVMInstance.obj
 0002:000001d4       ??_C@_0CH@KAGNBCII@?$FLINFO?$FN?3?5?5?5?5?5javaAccessBridgeWin@ 100081d4     AccessBridgeJavaVMInstance.obj
 0002:000001fc       ??_C@_0CC@NKGMANMJ@?$FLINFO?$FN?3?5In?5findAccessBridgeWind@ 100081fc     AccessBridgeJavaVMInstance.obj
 0002:00000220       ??_C@_0CK@NBPNOPCH@?$FLINFO?$FN?3?5In?5findABJavaInstanceFr@ 10008220     AccessBridgeJavaVMInstance.obj
 0002:00000250       ??_7exception@std@@6B@     10008250     AccessBridgeMessageQueue.obj
 0002:00000258       ??_C@_0BC@EOODALEL@Unknown?5exception@ 10008258     AccessBridgeMessageQueue.obj
 0002:00000270       ??_7bad_alloc@std@@6B@     10008270     AccessBridgeMessageQueue.obj
 0002:00000278       ??_C@_0P@GHFPNOJB@bad?5allocation@ 10008278     AccessBridgeMessageQueue.obj
 0002:00000288       ??_C@_0CN@EPCNBBKD@?$FLINFO?$FN?3?5?5?5in?5AccessBridgeMessag@ 10008288     AccessBridgeMessageQueue.obj
 0002:000002b8       ??_C@_0BM@FHOEMINC@?$FLINFO?$FN?3?5?5?5?5?5queue?5size?5?$DN?5?$CFd@ 100082b8     AccessBridgeMessageQueue.obj
 0002:000002d4       ??_C@_0DF@PKPPNDEN@?$FLWARN?$FN?3?5?5?5?5?5queue?5was?5locked?$DL?5r@ 100082d4     AccessBridgeMessageQueue.obj
 0002:0000030c       ??_C@_0CF@CAPEOLCL@?$FLINFO?$FN?3?5?5?5?5?5adding?5element?5to?5q@ 1000830c     AccessBridgeMessageQueue.obj
 0002:00000334       ??_C@_0DL@IILCMNMG@?$FLINFO?$FN?3?5?5?5?5?5returning?5from?5Acce@ 10008334     AccessBridgeMessageQueue.obj
 0002:00000370       ??_C@_0DA@NHLJEKKG@?$FLINFO?$FN?3?5?5?5in?5AccessBridgeMessag@ 10008370     AccessBridgeMessageQueue.obj
 0002:000003a0       ??_C@_0CJ@FBOCEMKO@?$FLINFO?$FN?3?5?5?5?5?5removing?5element?5fr@ 100083a0     AccessBridgeMessageQueue.obj
 0002:000003cc       ??_C@_0DO@NEJIEHGM@?$FLINFO?$FN?3?5?5?5?5?5returning?5from?5Acce@ 100083cc     AccessBridgeMessageQueue.obj
 0002:0000040c       ??_C@_0BM@BIAOFPJG@AccessBridge?9FromJava?9Hello@ 1000840c     AccessBridgeMessages.obj
 0002:00000428       ??_C@_0BP@OELHMMDF@AccessBridge?9FromWindows?9Hello@ 10008428     AccessBridgeMessages.obj
 0002:00000448       ??_C@_0DG@FAIBADKG@?$AN?6AccessBridgeWindowsEntryPoint@ 10008448     AccessBridgeWindowsEntryPoints.obj
 0002:00000480       ??_C@_0BG@GGFIABLO@windows_access_bridge@ 10008480     WinAccessBridge.obj
 0002:00000498       ??_C@_0BL@GLCNGDJJ@?$FLINFO?$FN?3?5DLL_PROCESS_ATTACH@ 10008498     WinAccessBridge.obj
 0002:000004b8       ??_C@_0EG@HHOMJPNP@?$FLINFO?$FN?3?5?$CK?$CK?$CK?5AccessBridgeDialogP@ 100084b8     WinAccessBridge.obj
 0002:00000500       ??_C@_0CP@LHINEKAP@?$FLINFO?$FN?3?5AccessBridgeDialogProc?5@ 10008500     WinAccessBridge.obj
 0002:00000530       ??_C@_0EH@MDELPMEJ@?$FLINFO?$FN?3?5AccessBridgeDialogProc?5@ 10008530     WinAccessBridge.obj
 0002:00000578       ??_C@_0DP@HBEMDAPF@?$FLINFO?$FN?3?5AccessBridgeDialogProc?5@ 10008578     WinAccessBridge.obj
 0002:000005b8       ??_C@_0EH@MPLEACPJ@?$FLINFO?$FN?3?5AccessBridgeDialogProc?5@ 100085b8     WinAccessBridge.obj
 0002:00000600       ??_C@_0EG@GGGHDKAD@?$FLINFO?$FN?3?5?$CK?$CK?$CK?$CK?$CK?5AccessBridgeDialo@ 10008600     WinAccessBridge.obj
 0002:00000648       ??_C@_0DE@BGNNIIOB@?$FLINFO?$FN?3?5?5?5javaVMs?5chain?5in?5use?0@ 10008648     WinAccessBridge.obj
 0002:0000067c       ??_C@_0CC@NEJJLLGC@?$FLINFO?$FN?3?5?5?5calling?5javaVMDestroy@ 1000867c     WinAccessBridge.obj
 0002:000006a0       ??_C@_0FG@BHPCMIAO@?$FLINFO?$FN?3?5AccessBridgeDialogProc?5@ 100086a0     WinAccessBridge.obj
 0002:000006f8       ??_C@_0BN@FIPGEIKI@?$FLINFO?$FN?3?5WinAccessBridge?5ctor@ 100086f8     WinAccessBridge.obj
 0002:00000718       ??_C@_0DE@JFKNENGC@?$FLINFO?$FN?3?5?$CK?$CK?$CK?$CK?$CKin?5WinAccessBridge@ 10008718     WinAccessBridge.obj
 0002:0000074c       ??_C@_0CG@EDMKMONP@?$FLINFO?$FN?3?5?5?5telling?5?$CFp?5we?8re?5goin@ 1000874c     WinAccessBridge.obj
 0002:00000774       ??_C@_0DB@CFPLAPDG@?$FLINFO?$FN?3?5?5?5finished?5telling?5JVMs@ 10008774     WinAccessBridge.obj
 0002:000007a8       ??_C@_0EE@GBJFCFOA@?$FLINFO?$FN?3?5?5?5finished?5deleting?5eve@ 100087a8     WinAccessBridge.obj
 0002:000007ec       ??_C@_0BP@EBFMIPOK@?$FLINFO?$FN?3?5GOODBYE?5CRUEL?5WORLD?4?4?4@ 100087ec     WinAccessBridge.obj
 0002:0000080c       ??_C@_0BJ@LMONFDOG@ACCESSBRIDGESTATUSWINDOW@ 1000880c     WinAccessBridge.obj
 0002:00000828       ??_C@_0DN@NNELAOKC@?$FLINFO?$FN?3?5in?5WinAccessBridge?3?3ren@ 10008828     WinAccessBridge.obj
 0002:00000868       ??_C@_0CJ@LMLGKPGD@?$FLINFO?$FN?3?5?5?5Setting?5Java?5event?5ma@ 10008868     WinAccessBridge.obj
 0002:00000894       ??_C@_0DC@IJKHOBEO@?$FLINFO?$FN?3?5?5?5Setting?5Accessibility@ 10008894     WinAccessBridge.obj
 0002:000008c8       ??_C@_0DN@ECLBFGAO@?$FLERROR?$FN?3?5Failed?5to?5initiate?5IPC@ 100088c8     WinAccessBridge.obj
 0002:00000908       ??_C@_0DG@OEMNKFJP@?$FLINFO?$FN?3?5?5?5Success?$CB?$CB?5?5We?5rendezv@ 10008908     WinAccessBridge.obj
 0002:00000940       ??_C@_0DK@BLMJEFJH@?$FLERROR?$FN?3?5sending?5memory?5package@ 10008940     WinAccessBridge.obj
 0002:0000097c       ??_C@_0DC@BABNPCOM@?$FLINFO?$FN?3?5?5in?5WinAccessBridge?3?3qu@ 1000897c     WinAccessBridge.obj
 0002:000009b0       ??_C@_0DE@NOAFOCML@?$FLINFO?$FN?3?5in?5WinAccessBridge?3?3rec@ 100089b0     WinAccessBridge.obj
 0002:000009e4       ??_C@_0BM@KNOOFOHJ@?$FLINFO?$FN?3?5?5dequeueing?5message@ 100089e4     WinAccessBridge.obj
 0002:00000a00       ??_C@_0CD@GBHFIMOB@?$FLERROR?$FN?3?5Queue?5seems?5to?5be?5brok@ 10008a00     WinAccessBridge.obj
 0002:00000a24       ??_C@_0CA@LFELFFDM@?$FLINFO?$FN?3?5?5found?5one?$DL?5sending?5it?$CB@ 10008a24     WinAccessBridge.obj
 0002:00000a44       ??_C@_0BP@ENBFDBDP@?$FLWARN?$FN?3?5?5?5ODD?4?4?4?5element?5?$DN?$DN?50?$CB@ 10008a44     WinAccessBridge.obj
 0002:00000a64       ??_C@_0CP@OIAJKCPF@?$FLWARN?$FN?3?5?5Queue?5in?5use?0?5will?5try@ 10008a64     WinAccessBridge.obj
 0002:00000a94       ??_C@_0DH@KAJCMPPF@?$FLWARN?$FN?3?5?5unable?5to?5dequeue?5mess@ 10008a94     WinAccessBridge.obj
 0002:00000acc       ??_C@_0CO@KCIANNAF@?$FLINFO?$FN?3?5PreProcessing?5package?5s@ 10008acc     WinAccessBridge.obj
 0002:00000b00       ??_C@_0EF@DFMGOCJF@?$FLERROR?$FN?3?5?5?5processing?5FAILED?$CB?$CB?5@ 10008b00     WinAccessBridge.obj
 0002:00000b48       ??_C@_0CL@HBCKEPEE@?$FLINFO?$FN?3?5?5?5?5package?5preprocessin@ 10008b48     WinAccessBridge.obj
 0002:00000b74       ??_C@_0DM@CCADHAH@?$FLINFO?$FN?3?5WinAccessBridge?3?3Proces@ 10008b74     WinAccessBridge.obj
 0002:00000bb0       ??_C@_0CI@KAACKIJC@?$FLINFO?$FN?3?5?5?5?5type?5?$DN?$DN?5cJavaShutdow@ 10008bb0     WinAccessBridge.obj
 0002:00000bd8       ??_C@_0CE@KGDIDFJM@?$FLINFO?$FN?3?5?5?5?5event?5callback?5compl@ 10008bd8     WinAccessBridge.obj
 0002:00000bfc       ??_C@_0BI@MGOIGNJM@?$FLINFO?$FN?3?5?5?5?5event?5fired?$CB@ 10008bfc     WinAccessBridge.obj
 0002:00000c18       ??_C@_0EC@JELBKKLB@?$FLERROR?$FN?3?5?5?5?5processing?5FAILED?$CB?$CB@ 10008c18     WinAccessBridge.obj
 0002:00000c5c       ??_C@_0CM@OIHFPHBP@?$FLINFO?$FN?3?5?5?5?5begin?5callback?5to?5AT@ 10008c5c     WinAccessBridge.obj
 0002:00000c88       ??_C@_0EB@PCOLNIOI@?$FLERROR?$FN?3?5?5?5processing?5FAILED?$CB?$CB?5@ 10008c88     WinAccessBridge.obj
 0002:00000cd0       ??_C@_0EG@DADDGPDA@?$FLERROR?$FN?3?5?5?5?5processing?5FAILED?$CB?$CB@ 10008cd0     WinAccessBridge.obj
 0002:00000d18       ??_C@_0CI@PMGDCMNI@?$FLINFO?$FN?3?5?5?5?5package?5processing?5c@ 10008d18     WinAccessBridge.obj
 0002:00000d40       ??_C@_0DD@EDMANGOO@?$FLINFO?$FN?3?5?$CK?$CK?$CK?$CK?$CK?5WinAccessBridge?3?3@ 10008d40     WinAccessBridge.obj
 0002:00000d74       ??_C@_0CP@IIHJFGGB@?$FLINFO?$FN?3?5?5?5data?5structures?5succe@ 10008d74     WinAccessBridge.obj
 0002:00000da4       ??_C@_0DB@JABMCGEJ@?$FLERROR?$FN?3?5couldn?8t?5find?5matching@ 10008da4     WinAccessBridge.obj
 0002:00000dd8       ??_C@_0DD@BOICBNBL@?$FLINFO?$FN?3?5WinAccessBridge?3?3releas@ 10008dd8     WinAccessBridge.obj
 0002:00000e0c       ??_C@_0CO@GDCOMIDN@?$FLINFO?$FN?3?5WinAccessBridge?3?3getVer@ 10008e0c     WinAccessBridge.obj
 0002:00000e40       ??_C@_0IH@JNMBAFNI@?$FLINFO?$FN?3?5?5?5VMversion?3?5?$CFls?6?5?5?5?5?5?5@ 10008e40     WinAccessBridge.obj
 0002:00000ec8       ??_C@_0CJ@MFBANPLF@?$FLINFO?$FN?3?5In?5WinAccessBridge?3?3isJ@ 10008ec8     WinAccessBridge.obj
 0002:00000ef4       ??_C@_0CK@OIADIKJK@?$FLINFO?$FN?3?5WinAccessBridge?3?3isJava@ 10008ef4     WinAccessBridge.obj
 0002:00000f20       ??_C@_0CN@JBJBEHML@?$FLINFO?$FN?3?5WinAccessBridge?3?3isSame@ 10008f20     WinAccessBridge.obj
 0002:00000f50       ??_C@_0EF@JHJAECO@?$FLINFO?$FN?3?5?5?5WinAccessBridge?3?3isSa@ 10008f50     WinAccessBridge.obj
 0002:00000f98       ??_C@_0EL@EGCPHNBB@?$FLINFO?$FN?3?5?5?5WinAccessBridge?3?3isSa@ 10008f98     WinAccessBridge.obj
 0002:00000fe8       ??_C@_0FE@JNIGOBOL@?$FLERROR?$FN?3?5?5?5WinAccessBridge?3?3isS@ 10008fe8     WinAccessBridge.obj
 0002:0000103c       ??_C@_0DM@KHCMPGEG@?$FLINFO?$FN?3?5WinAccessBridge?3?3getAcc@ 1000903c     WinAccessBridge.obj
 0002:00001078       ??_C@_0DA@KDJKNLAN@?$FLINFO?$FN?3?5?5?5?5?5current?9?$DOvmID?5?$DN?5?$CFX?0@ 10009078     WinAccessBridge.obj
 0002:000010a8       ??_C@_0CJ@HIABIFFO@?$FLINFO?$FN?3?5?5?5?5?5pkg?9?$DOrAccessibleCon@ 100090a8     WinAccessBridge.obj
 0002:000010d4       ??_C@_0DJ@FFBPMFOM@?$FLERROR?$FN?3?5getAccessibleContextFr@ 100090d4     WinAccessBridge.obj
 0002:00001110       ??_C@_0DO@IIGOCPCC@?$FLERROR?$FN?3?5getAccessibleContextFr@ 10009110     WinAccessBridge.obj
 0002:00001150       ??_C@_0DL@KEEIEGBJ@?$FLINFO?$FN?3?5?5?5in?5WinAccessBridge?3?3g@ 10009150     WinAccessBridge.obj
 0002:0000118c       ??_C@_0DK@JJIBFDBC@?$FLINFO?$FN?3?5WinAccessBridge?3?3getHWN@ 1000918c     WinAccessBridge.obj
 0002:000011c8       ??_C@_0EA@FHJPOEHJ@?$FLINFO?$FN?3?5WinAccessBridge?3?3getAcc@ 100091c8     WinAccessBridge.obj
 0002:00001208       ??_C@_0EB@HKEAOAKG@?$FLINFO?$FN?3?5WinAccessBridge?3?3getAcc@ 10009208     WinAccessBridge.obj
 0002:0000124c       ??_C@_0DM@JJBOABOC@?$FLINFO?$FN?3?5WinAccessBridge?3?3getAcc@ 1000924c     WinAccessBridge.obj
 0002:00001288       ??_C@_0JA@MODCAACP@?$FLINFO?$FN?3?5?5?5name?3?5?$CFls?6?5?5?5?5?5?5?5?5?5?5d@ 10009288     WinAccessBridge.obj
 0002:00001318       ??_C@_0ED@KCHDBBOB@?$FLINFO?$FN?3?5WinAccessBridge?3?3getAcc@ 10009318     WinAccessBridge.obj
 0002:00001360       ??_C@_0EA@MDGJLODH@?$FLINFO?$FN?3?5WinAccessBridge?3?3getAcc@ 10009360     WinAccessBridge.obj
 0002:000013a0       ??_C@_0EC@NLPKJMMJ@?$FLINFO?$FN?3?5?$CD?$CD?$CD?$CD?$CD?5WinAccessBridge?3?3@ 100093a0     WinAccessBridge.obj
 0002:000013e8       ??_C@_0EC@FNKONEFN@?$FLINFO?$FN?3?5?5?5?$CD?$CD?$CD?$CD?$CD?5WinAccessBridge@ 100093e8     WinAccessBridge.obj
 0002:00001430       ??_C@_0EA@GPGOILHN@?$FLERROR?$FN?3?5?5?5?$CD?$CD?$CD?$CD?$CD?5WinAccessBridg@ 10009430     WinAccessBridge.obj
 0002:00001470       ??_C@_0EO@GIFIOBJO@?$FLINFO?$FN?3?5?$CD?$CD?$CD?$CD?$CD?5WinAccessBridge?3?3@ 10009470     WinAccessBridge.obj
 0002:000014c0       ??_C@_0DK@FPHEFKPF@?$FLINFO?$FN?3?5?5?5XXXX?5pkg?9?$DOrTableCellI@ 100094c0     WinAccessBridge.obj
 0002:00001500       ??_C@_0EG@CFNEHAJF@?$FLINFO?$FN?3?5?5?5?$CD?$CD?$CD?$CD?$CD?5WinAccessBridge@ 10009500     WinAccessBridge.obj
 0002:00001548       ??_C@_0EE@DMEKGPAL@?$FLERROR?$FN?3?5?5?5?$CD?$CD?$CD?$CD?$CD?5WinAccessBridg@ 10009548     WinAccessBridge.obj
 0002:00001590       ??_C@_0ED@PHPOFILJ@?$FLINFO?$FN?3?5?$CD?$CD?$CD?$CD?$CD?5WinAccessBridge?3?3@ 10009590     WinAccessBridge.obj
 0002:000015d8       ??_C@_0EH@MMAIEADN@?$FLINFO?$FN?3?5?5?5?$CD?$CD?$CD?$CD?$CD?5WinAccessBridge@ 100095d8     WinAccessBridge.obj
 0002:00001620       ??_C@_0EF@IGPDOLOH@?$FLERROR?$FN?3?5?5?5?$CD?$CD?$CD?$CD?$CD?5WinAccessBridg@ 10009620     WinAccessBridge.obj
 0002:00001668       ??_C@_0EG@HBMADODM@?$FLINFO?$FN?3?5?$CD?$CD?$CD?$CD?$CD?5WinAccessBridge?3?3@ 10009668     WinAccessBridge.obj
 0002:000016b0       ??_C@_0EK@DJMDCCLK@?$FLINFO?$FN?3?5?5?5?$CD?$CD?$CD?$CD?$CD?5WinAccessBridge@ 100096b0     WinAccessBridge.obj
 0002:00001700       ??_C@_0EI@CELDDCKP@?$FLERROR?$FN?3?5?5?5?$CD?$CD?$CD?$CD?$CD?5WinAccessBridg@ 10009700     WinAccessBridge.obj
 0002:00001748       ??_C@_0EM@IIFJHKCG@?$FLINFO?$FN?3?5?$CD?$CD?$CD?$CD?$CD?5WinAccessBridge?3?3@ 10009748     WinAccessBridge.obj
 0002:00001798       ??_C@_0EM@JPIPIDPC@?$FLINFO?$FN?3?5?5?5?$CD?$CD?$CD?$CD?$CD?5WinAccessBridge@ 10009798     WinAccessBridge.obj
 0002:000017e8       ??_C@_0EK@IGPCFPOI@?$FLERROR?$FN?3?5?5?5?$CD?$CD?$CD?$CD?$CD?5WinAccessBridg@ 100097e8     WinAccessBridge.obj
 0002:00001838       ??_C@_0EP@ICKKLPNA@?$FLINFO?$FN?3?5?$CD?$CD?$CD?$CD?$CD?5WinAccessBridge?3?3@ 10009838     WinAccessBridge.obj
 0002:00001888       ??_C@_0EP@PJFHLMKB@?$FLINFO?$FN?3?5?5?5?$CD?$CD?$CD?$CD?$CD?5WinAccessBridge@ 10009888     WinAccessBridge.obj
 0002:000018d8       ??_C@_0EN@FJIGOJNI@?$FLERROR?$FN?3?5?5?5?$CD?$CD?$CD?$CD?$CD?5WinAccessBridg@ 100098d8     WinAccessBridge.obj
 0002:00001928       ??_C@_0EL@KJJDJJDB@?$FLINFO?$FN?3?5?$CD?$CD?$CD?$CD?$CD?5WinAccessBridge?3?3@ 10009928     WinAccessBridge.obj
 0002:00001978       ??_C@_0EP@DHAGNOBO@?$FLINFO?$FN?3?5?5?5?$CD?$CD?$CD?$CD?$CD?5WinAccessBridge@ 10009978     WinAccessBridge.obj
 0002:000019c8       ??_C@_0EN@IFAFODLF@?$FLERROR?$FN?3?5?5?5?$CD?$CD?$CD?$CD?$CD?5WinAccessBridg@ 100099c8     WinAccessBridge.obj
 0002:00001a18       ??_C@_0EE@LHHJOBIL@?$FLINFO?$FN?3?5?$CD?$CD?$CD?$CD?$CD?5WinAccessBridge?3?3@ 10009a18     WinAccessBridge.obj
 0002:00001a60       ??_C@_0EI@LCHMKLCB@?$FLINFO?$FN?3?5?5?5?$CD?$CD?$CD?$CD?$CD?5WinAccessBridge@ 10009a60     WinAccessBridge.obj
 0002:00001aa8       ??_C@_0EG@PCFFNJPM@?$FLERROR?$FN?3?5?5?5?$CD?$CD?$CD?$CD?$CD?5WinAccessBridg@ 10009aa8     WinAccessBridge.obj
 0002:00001af0       ??_C@_0EH@BHDKFALD@?$FLINFO?$FN?3?5?$CD?$CD?$CD?$CD?$CD?5WinAccessBridge?3?3@ 10009af0     WinAccessBridge.obj
 0002:00001b38       ??_C@_0EL@HPJEOBAF@?$FLINFO?$FN?3?5?5?5?$CD?$CD?$CD?$CD?$CD?5WinAccessBridge@ 10009b38     WinAccessBridge.obj
 0002:00001b88       ??_C@_0EJ@EFJNHGOC@?$FLERROR?$FN?3?5?5?5?$CD?$CD?$CD?$CD?$CD?5WinAccessBridg@ 10009b88     WinAccessBridge.obj
 0002:00001bd8       ??_C@_0EO@FKPIEILP@?$FLINFO?$FN?3?5?$CD?$CD?$CD?$CD?$CD?5WinAccessBridge?3?3@ 10009bd8     WinAccessBridge.obj
 0002:00001c28       ??_C@_0FC@IJCKDOEL@?$FLINFO?$FN?3?5?5?5?$CD?$CD?$CD?$CD?$CD?5WinAccessBridge@ 10009c28     WinAccessBridge.obj
 0002:00001c80       ??_C@_0FA@EEJJLKOB@?$FLERROR?$FN?3?5?5?5?$CD?$CD?$CD?$CD?$CD?5WinAccessBridg@ 10009c80     WinAccessBridge.obj
 0002:00001cd0       ??_C@_0EH@FBPCBBDM@?$FLINFO?$FN?3?5?$CD?$CD?$CD?$CD?$CD?5WinAccessBridge?3?3@ 10009cd0     WinAccessBridge.obj
 0002:00001d18       ??_C@_0EL@MCFEFCEP@?$FLINFO?$FN?3?5?5?5?$CD?$CD?$CD?$CD?$CD?5WinAccessBridge@ 10009d18     WinAccessBridge.obj
 0002:00001d68       ??_C@_0EJ@OEGCIAEN@?$FLERROR?$FN?3?5?5?5?$CD?$CD?$CD?$CD?$CD?5WinAccessBridg@ 10009d68     WinAccessBridge.obj
 0002:00001db8       ??_C@_0EK@MEPJJMEA@?$FLINFO?$FN?3?5?$CD?$CD?$CD?$CD?$CD?5WinAccessBridge?3?3@ 10009db8     WinAccessBridge.obj
 0002:00001e08       ??_C@_0EO@KBJAHINP@?$FLINFO?$FN?3?5?5?5?$CD?$CD?$CD?$CD?$CD?5WinAccessBridge@ 10009e08     WinAccessBridge.obj
 0002:00001e58       ??_C@_0EM@FBMEIFEO@?$FLERROR?$FN?3?5?5?5?$CD?$CD?$CD?$CD?$CD?5WinAccessBridg@ 10009e58     WinAccessBridge.obj
 0002:00001ea8       ??_C@_0EH@PCGFNBKC@?$FLINFO?$FN?3?5?$CD?$CD?$CD?$CD?$CD?5WinAccessBridge?3?3@ 10009ea8     WinAccessBridge.obj
 0002:00001ef0       ??_C@_0EB@EHNAMLGG@?$FLINFO?$FN?3?5?5?5?$CD?$CD?$CD?$CD?$CD?5WinAccessBridge@ 10009ef0     WinAccessBridge.obj
 0002:00001f34       ??_C@_0DP@JGIKFGJD@?$FLERROR?$FN?3?5?5?5?$CD?$CD?$CD?$CD?$CD?5WinAccessBridg@ 10009f34     WinAccessBridge.obj
 0002:00001f78       ??_C@_0EK@CBKGBNFB@?$FLINFO?$FN?3?5?$CD?$CD?$CD?$CD?$CD?5WinAccessBridge?3?3@ 10009f78     WinAccessBridge.obj
 0002:00001fc8       ??_C@_0EE@HJIACDJB@?$FLINFO?$FN?3?5?5?5?$CD?$CD?$CD?$CD?$CD?5WinAccessBridge@ 10009fc8     WinAccessBridge.obj
 0002:00002010       ??_C@_0EC@HJIAKIIH@?$FLERROR?$FN?3?5?5?5?$CD?$CD?$CD?$CD?$CD?5WinAccessBridg@ 1000a010     WinAccessBridge.obj
 0002:00002058       ??_C@_0EP@OKKBNNPD@?$FLINFO?$FN?3?5?$CD?$CD?$CD?$CD?$CD?5WinAccessBridge?3?3@ 1000a058     WinAccessBridge.obj
 0002:000020a8       ??_C@_0ED@CBAGECAG@?$FLINFO?$FN?3?5?5?5?$CD?$CD?$CD?$CD?$CD?5WinAccessBridge@ 1000a0a8     WinAccessBridge.obj
 0002:000020f0       ??_C@_0EB@NLKCNKIL@?$FLERROR?$FN?3?5?5?5?$CD?$CD?$CD?$CD?$CD?5WinAccessBridg@ 1000a0f0     WinAccessBridge.obj
 0002:00002138       ??_C@_0EE@OCGNGPOA@?$FLINFO?$FN?3?5?$CD?$CD?$CD?$CD?$CD?5WinAccessBridge?3?3@ 1000a138     WinAccessBridge.obj
 0002:00002180       ??_C@_0ED@KBOKJBJ@?$FLINFO?$FN?3?5?5?5?$CD?$CD?$CD?$CD?$CD?5pkg?9?$DOrAccessibl@ 1000a180     WinAccessBridge.obj
 0002:000021c8       ??_C@_0EE@MLCJPFKH@?$FLINFO?$FN?3?5?5?5?$CD?$CD?$CD?$CD?$CD?5WinAccessBridge@ 1000a1c8     WinAccessBridge.obj
 0002:00002210       ??_C@_0EC@ONHLHLKJ@?$FLERROR?$FN?3?5?5?5?$CD?$CD?$CD?$CD?$CD?5WinAccessBridg@ 1000a210     WinAccessBridge.obj
 0002:00002258       ??_C@_0EC@FGNNKNB@?$FLINFO?$FN?3?5?$CD?$CD?$CD?$CD?$CD?5WinAccessBridge?3?3@ 1000a258     WinAccessBridge.obj
 0002:0000229c       ??_C@_0CN@CIJKLIHC@?$FLINFO?$FN?3?5?5?5?$CD?$CD?$CD?$CD?$CD?5hypertextInfo?4l@ 1000a29c     WinAccessBridge.obj
 0002:000022d0       ??_C@_0EC@GJFIBKBJ@?$FLINFO?$FN?3?5?5?5?$CD?$CD?$CD?$CD?$CD?5WinAccessBridge@ 1000a2d0     WinAccessBridge.obj
 0002:00002318       ??_C@_0EA@ENIAHHMF@?$FLERROR?$FN?3?5?5?5?$CD?$CD?$CD?$CD?$CD?5WinAccessBridg@ 1000a318     WinAccessBridge.obj
 0002:00002358       ??_C@_0DM@HHDHADBA@?$FLINFO?$FN?3?5WinAccessBridge?3?3activa@ 1000a358     WinAccessBridge.obj
 0002:00002398       ??_C@_0GC@OOPIFCLD@?$FLERROR?$FN?3?5?5WinAccessBridge?3?3acti@ 1000a398     WinAccessBridge.obj
 0002:00002400       ??_C@_0ED@PBOHFCGF@?$FLINFO?$FN?3?5?$CD?$CD?$CD?$CD?$CD?5WinAccessBridge?3?3@ 1000a400     WinAccessBridge.obj
 0002:00002444       ??_C@_0CJ@CHHBPBDA@?$FLINFO?$FN?3?5?5?5?$CD?$CD?$CD?$CD?$CD?5hypetext?5link?5c@ 1000a444     WinAccessBridge.obj
 0002:00002470       ??_C@_0EG@OFFPNIFM@?$FLINFO?$FN?3?5?5?$CD?$CD?$CD?$CD?$CD?5WinAccessBridge?3@ 1000a470     WinAccessBridge.obj
 0002:000024b8       ??_C@_0EF@CJEMCIKC@?$FLERROR?$FN?3?5?5?5?$CD?$CD?$CD?$CD?$CD?5WinAccessBridg@ 1000a4b8     WinAccessBridge.obj
 0002:00002500       ??_C@_0EE@NGLHNPAI@?$FLINFO?$FN?3?5?$CD?$CD?$CD?$CD?$CD?5WinAccessBridge?3?3@ 1000a500     WinAccessBridge.obj
 0002:00002544       ??_C@_0CD@FAKLHPNN@?$FLINFO?$FN?3?5?5?5?$CD?$CD?$CD?$CD?$CD?5pkg?9?$DOrSuccess?5?$DN@ 1000a544     WinAccessBridge.obj
 0002:00002568       ??_C@_0ED@CLMPFLBE@?$FLERROR?$FN?3?5?5?5?$CD?$CD?$CD?$CD?$CD?5WinAccessBridg@ 1000a568     WinAccessBridge.obj
 0002:000025b0       ??_C@_0EC@DJBOOIDG@?$FLERROR?$FN?3?5?5?$CD?$CD?$CD?$CD?$CD?5WinAccessBridge@ 1000a5b0     WinAccessBridge.obj
 0002:000025f8       ??_C@_0EH@NNKMHKPC@?$FLINFO?$FN?3?5?$CD?$CD?$CD?$CD?$CD?5WinAccessBridge?3?3@ 1000a5f8     WinAccessBridge.obj
 0002:00002640       ??_C@_0CJ@LGNOCJK@?$FLINFO?$FN?3?5?5?5?$CD?$CD?$CD?$CD?$CD?5hypetext?5link?5i@ 1000a640     WinAccessBridge.obj
 0002:00002670       ??_C@_0EM@KCINDCOI@?$FLINFO?$FN?3?5?5?5?$CD?$CD?$CD?$CD?$CD?5WinAccessBridge@ 1000a670     WinAccessBridge.obj
 0002:000026c0       ??_C@_0EI@IEJDJKBK@?$FLERROR?$FN?5?5?$CD?$CD?$CD?$CD?$CD?5WinAccessBridge?3@ 1000a6c0     WinAccessBridge.obj
 0002:00002708       ??_C@_0EC@DDOOALIF@?$FLINFO?$FN?3?5?$CD?$CD?$CD?$CD?$CD?5WinAccessBridge?3?3@ 1000a708     WinAccessBridge.obj
 0002:00002750       ??_C@_0EE@CCNHBKL@?$FLINFO?$FN?3?5?$CD?$CD?$CD?$CD?$CD?5WinAccessBridge?3?3@ 1000a750     WinAccessBridge.obj
 0002:00002794       ??_C@_0DC@GOKFJHHA@?$FLINFO?$FN?3?5?5?5?$CD?$CD?$CD?$CD?$CD?5keyBindings?4key@ 1000a794     WinAccessBridge.obj
 0002:000027c8       ??_C@_0KM@PICKCJIM@?$FLINFO?$FN?3?5?5?5Key?5Binding?5?$CD?5?$CFd?5?5?5?5?5@ 1000a7c8     WinAccessBridge.obj
 0002:00002878       ??_C@_0EE@LGIDNFJF@?$FLINFO?$FN?3?5?5?5?$CD?$CD?$CD?$CD?$CD?5WinAccessBridge@ 1000a878     WinAccessBridge.obj
 0002:000028c0       ??_C@_0EB@PIGLELIJ@?$FLINFO?$FN?3?5?5?5?$CD?$CD?$CD?$CD?$CD?5WinAccessBridge@ 1000a8c0     WinAccessBridge.obj
 0002:00002904       ??_C@_0DO@OLOBAIEE@?$FLINFO?$FN?3?5?$CD?$CD?$CD?$CD?$CD?5WinAccessBridge?3?3@ 1000a904     WinAccessBridge.obj
 0002:00002944       ??_C@_0CG@JNBKIMJN@?$FLINFO?$FN?3?5?5?5?$CD?$CD?$CD?$CD?$CD?5icons?4iconsCoun@ 1000a944     WinAccessBridge.obj
 0002:0000296c       ??_C@_0DO@JGGAAEEG@?$FLINFO?$FN?3?5?5?5?$CD?$CD?$CD?$CD?$CD?5WinAccessBridge@ 1000a96c     WinAccessBridge.obj
 0002:000029ac       ??_C@_0DM@PHFGBDGG@?$FLERROR?$FN?3?5?5?5?$CD?$CD?$CD?$CD?$CD?5WinAccessBridg@ 1000a9ac     WinAccessBridge.obj
 0002:000029e8       ??_C@_0EA@BGCCBFCM@?$FLINFO?$FN?3?5?$CD?$CD?$CD?$CD?$CD?5WinAccessBridge?3?3@ 1000a9e8     WinAccessBridge.obj
 0002:00002a28       ??_C@_0CK@COBILBN@?$FLINFO?$FN?3?5?5?5?$CD?$CD?$CD?$CD?$CD?5actions?4actions@ 1000aa28     WinAccessBridge.obj
 0002:00002a58       ??_C@_0EA@EKDNLNJA@?$FLINFO?$FN?3?5?5?5?$CD?$CD?$CD?$CD?$CD?5WinAccessBridge@ 1000aa58     WinAccessBridge.obj
 0002:00002a98       ??_C@_0DO@HNCGODDL@?$FLERROR?$FN?3?5?5?5?$CD?$CD?$CD?$CD?$CD?5WinAccessBridg@ 1000aa98     WinAccessBridge.obj
 0002:00002ad8       ??_C@_0EB@PGNJAJIF@?$FLINFO?$FN?3?5WinAccessBridge?3?3doAcce@ 1000aad8     WinAccessBridge.obj
 0002:00002b20       ??_C@_0FL@LJNDNJAB@?$FLERROR?$FN?3?5?5?5WinAccessBridge?3?3doA@ 1000ab20     WinAccessBridge.obj
 0002:00002b7c       ??_C@_0DL@JCIKLICA@?$FLINFO?$FN?3?5WinAccessBridge?3?3setTex@ 1000ab7c     WinAccessBridge.obj
 0002:00002bb8       ??_C@_0DD@CAEDECNM@?$FLINFO?$FN?3?5WinAccessBridge?3?3getPar@ 1000abb8     WinAccessBridge.obj
 0002:00002bf0       ??_C@_0FE@FILBCBC@?$FLINFO?$FN?3?5?5?5pkg?9?$DOvmID?3?5?$CFX?5?5?5?5?5?5?5?5@ 1000abf0     WinAccessBridge.obj
 0002:00002c44       ??_C@_0CG@EPJKPFNH@?$FLINFO?$FN?3?5?5?5pkg?9?$DOrAccessibleConte@ 1000ac44     WinAccessBridge.obj
 0002:00002c6c       ??_C@_0DD@PJCACADD@?$FLINFO?$FN?3?5WinAccessBridge?3?3getTop@ 1000ac6c     WinAccessBridge.obj
 0002:00002ca0       ??_C@_0DL@DOMCMOCA@?$FLINFO?$FN?3?5WinAccessBridge?3?3getPar@ 1000aca0     WinAccessBridge.obj
 0002:00002cdc       ??_C@_0DA@NHDILDKL@?$FLINFO?$FN?3?5WinAccessBridge?3?3getObj@ 1000acdc     WinAccessBridge.obj
 0002:00002d0c       ??_C@_0DF@CJFEBMOH@?$FLINFO?$FN?3?5WinAccessBridge?3?3getAct@ 1000ad0c     WinAccessBridge.obj
 0002:00002d44       ??_C@_0DK@CBNGPLCC@?$FLINFO?$FN?3?5WinAccessBridge?3?3getVir@ 1000ad44     WinAccessBridge.obj
 0002:00002d80       ??_C@_0EK@LJJEDFEG@?$FLINFO?$FN?3?5?5?5?5?5WinAccessBridge?3?3ge@ 1000ad80     WinAccessBridge.obj
 0002:00002dcc       ??_C@_0CO@FBMJHILD@?$FLINFO?$FN?3?5WinAccessBridge?3?3reques@ 1000adcc     WinAccessBridge.obj
 0002:00002dfc       ??_C@_0DL@EHMNJADE@?$FLINFO?$FN?3?5?5?5?5?5WinAccessBridge?3?3se@ 1000adfc     WinAccessBridge.obj
 0002:00002e38       ??_C@_0EE@MACKKBMI@?$FLINFO?$FN?3?5?5?5?5?5WinAccessBridge?3?3ge@ 1000ae38     WinAccessBridge.obj
 0002:00002e7c       ??_C@_0DJ@MONFABKN@?$FLINFO?$FN?3?5WinAccessBridge?3?3getVis@ 1000ae7c     WinAccessBridge.obj
 0002:00002eb8       ??_C@_0DE@PJJKAOH@?$FLINFO?$FN?3?5WinAccessBridge?3?3getVis@ 1000aeb8     WinAccessBridge.obj
 0002:00002eec       ??_C@_0DG@FMHJPMAD@?$FLINFO?$FN?3?5WinAccessBridge?3?3setCar@ 1000aeec     WinAccessBridge.obj
 0002:00002f28       ??_C@_0ED@NHEGBLJF@?$FLINFO?$FN?3?5WinAccessBridge?3?3getAcc@ 1000af28     WinAccessBridge.obj
 0002:00002f70       ??_C@_0EK@DNDDFNHD@?$FLINFO?$FN?3?5?5?5charCount?3?5?$CFd?5?5?5?5?5?5?5?5@ 1000af70     WinAccessBridge.obj
 0002:00002fc0       ??_C@_0EA@DIFPCEIC@?$FLINFO?$FN?3?5WinAccessBridge?3?3getAcc@ 1000afc0     WinAccessBridge.obj
 0002:00003000       ??_C@_0EE@PALDCFAG@?$FLINFO?$FN?3?5WinAccessBridge?3?3getAcc@ 1000b000     WinAccessBridge.obj
 0002:00003048       ??_C@_0EF@HGMJALLO@?$FLINFO?$FN?3?5WinAccessBridge?3?3getAcc@ 1000b048     WinAccessBridge.obj
 0002:00003090       ??_C@_0DP@CLMLEHCN@?$FLINFO?$FN?3?5WinAccessBridge?3?3getAcc@ 1000b090     WinAccessBridge.obj
 0002:000030d0       ??_C@_0DK@FNDDJPBM@?$FLINFO?$FN?3?5WinAccessBridge?3?3getCar@ 1000b0d0     WinAccessBridge.obj
 0002:00003110       ??_C@_0ED@LPENFOEL@?$FLINFO?$FN?3?5WinAccessBridge?3?3getAcc@ 1000b110     WinAccessBridge.obj
 0002:00003158       ??_C@_0EC@MFICIOBI@?$FLINFO?$FN?3?5WinAccessBridge?3?3getAcc@ 1000b158     WinAccessBridge.obj
 0002:0000319c       ??_C@_0DM@NFGOCJPM@?$FLINFO?$FN?3?5WinAccessBridge?3?3addJav@ 1000b19c     WinAccessBridge.obj
 0002:000031d8       ??_C@_0DP@PIGNLFHB@?$FLINFO?$FN?3?5?5?5?9?$DOpkgType?5?$DN?5?$CFX?0?5event@ 1000b1d8     WinAccessBridge.obj
 0002:00003218       ??_C@_0EC@OKCIJGM@?$FLINFO?$FN?3?5in?5WinAccessBridge?3?3rem@ 1000b218     WinAccessBridge.obj
 0002:00003260       ??_C@_0EI@HMKIAPB@?$FLINFO?$FN?3?5in?5WinAccessBridge?3?3add@ 1000b260     WinAccessBridge.obj
 0002:000032a8       ??_C@_0DP@KFDABLNL@?$FLINFO?$FN?3?5?5?5?9?$DOpkgType?5?$DN?5?$CFX?0?5event@ 1000b2a8     WinAccessBridge.obj
 0002:000032e8       ??_C@_0EL@BFCCGHFN@?$FLINFO?$FN?3?5in?5WinAccessBridge?3?3rem@ 1000b2e8     WinAccessBridge.obj
 0002:00003338       ??_7type_info@@6B@         1000b338     MSVCRT:std_type_info_static.obj
 0002:0000333c       __pDefaultRawDllMain       1000b33c     MSVCRT:dll_dllmain.obj
 0002:0000333c       __pRawDllMain              1000b33c     MSVCRT:dll_dllmain.obj
 0002:0000334c       ??_7bad_array_new_length@std@@6B@ 1000b34c     MSVCRT:throw_bad_alloc.obj
 0002:00003354       ??_C@_0BF@KINCDENJ@bad?5array?5new?5length@ 1000b354     MSVCRT:throw_bad_alloc.obj
 0002:00003370       __load_config_used         1000b370     MSVCRT:loadcfg.obj
 0002:000034c0       ??_R4exception@std@@6B@    1000b4c0     AccessBridgeMessageQueue.obj
 0002:000034d4       ??_R3exception@std@@8      1000b4d4     AccessBridgeMessageQueue.obj
 0002:000034e4       ??_R2exception@std@@8      1000b4e4     AccessBridgeMessageQueue.obj
 0002:000034ec       ??_R1A@?0A@EA@exception@std@@8 1000b4ec     AccessBridgeMessageQueue.obj
 0002:00003508       ??_R4bad_alloc@std@@6B@    1000b508     AccessBridgeMessageQueue.obj
 0002:0000351c       ??_R3bad_alloc@std@@8      1000b51c     AccessBridgeMessageQueue.obj
 0002:0000352c       ??_R2bad_alloc@std@@8      1000b52c     AccessBridgeMessageQueue.obj
 0002:00003538       ??_R1A@?0A@EA@bad_alloc@std@@8 1000b538     AccessBridgeMessageQueue.obj
 0002:00003554       ??_R4type_info@@6B@        1000b554     MSVCRT:std_type_info_static.obj
 0002:00003568       ??_R3type_info@@8          1000b568     MSVCRT:std_type_info_static.obj
 0002:00003578       ??_R2type_info@@8          1000b578     MSVCRT:std_type_info_static.obj
 0002:00003580       ??_R1A@?0A@EA@type_info@@8 1000b580     MSVCRT:std_type_info_static.obj
 0002:0000359c       ??_R4bad_array_new_length@std@@6B@ 1000b59c     MSVCRT:throw_bad_alloc.obj
 0002:000035b0       ??_R3bad_array_new_length@std@@8 1000b5b0     MSVCRT:throw_bad_alloc.obj
 0002:000035c0       ??_R2bad_array_new_length@std@@8 1000b5c0     MSVCRT:throw_bad_alloc.obj
 0002:000035d0       ??_R1A@?0A@EA@bad_array_new_length@std@@8 1000b5d0     MSVCRT:throw_bad_alloc.obj
 0002:000035ec       ___safe_se_handler_table   1000b5ec     <linker-defined>
 0002:000035f0       ___volatile_metadata       1000b5f0     <linker-defined>
 0002:0000393c       ___rtc_iaa                 1000b93c     MSVCRT:initsect.obj
 0002:00003940       ___rtc_izz                 1000b940     MSVCRT:initsect.obj
 0002:00003944       ___rtc_taa                 1000b944     MSVCRT:initsect.obj
 0002:00003948       ___rtc_tzz                 1000b948     MSVCRT:initsect.obj
 0002:00003950       __CT??_R0?AVbad_alloc@std@@@8??0bad_alloc@std@@QAE@ABV01@@Z12 1000b950     AccessBridgeMessageQueue.obj
 0002:0000396c       __CT??_R0?AVexception@std@@@8??0exception@std@@QAE@ABV01@@Z12 1000b96c     AccessBridgeMessageQueue.obj
 0002:00003988       __TI2?AVbad_alloc@std@@    1000b988     AccessBridgeMessageQueue.obj
 0002:00003998       __CTA2?AVbad_alloc@std@@   1000b998     AccessBridgeMessageQueue.obj
 0002:00003a0c       __TI3?AVbad_array_new_length@std@@ 1000ba0c     MSVCRT:throw_bad_alloc.obj
 0002:00003a1c       __CTA3?AVbad_array_new_length@std@@ 1000ba1c     MSVCRT:throw_bad_alloc.obj
 0002:00003a2c       __CT??_R0?AVbad_array_new_length@std@@@8??0bad_array_new_length@std@@QAE@ABV01@@Z12 1000ba2c     MSVCRT:throw_bad_alloc.obj
 0002:000048b0       __IMPORT_DESCRIPTOR_KERNEL32 1000c8b0     kernel32:KERNEL32.dll
 0002:000048c4       __IMPORT_DESCRIPTOR_USER32 1000c8c4     user32:USER32.dll
 0002:000048d8       __IMPORT_DESCRIPTOR_VCRUNTIME140 1000c8d8     vcruntime:VCRUNTIME140.dll
 0002:000048ec       __IMPORT_DESCRIPTOR_api-ms-win-crt-string-l1-1-0 1000c8ec     ucrt:api-ms-win-crt-string-l1-1-0.dll
 0002:00004900       __IMPORT_DESCRIPTOR_api-ms-win-crt-stdio-l1-1-0 1000c900     ucrt:api-ms-win-crt-stdio-l1-1-0.dll
 0002:00004914       __IMPORT_DESCRIPTOR_api-ms-win-crt-environment-l1-1-0 1000c914     ucrt:api-ms-win-crt-environment-l1-1-0.dll
 0002:00004928       __IMPORT_DESCRIPTOR_api-ms-win-crt-heap-l1-1-0 1000c928     ucrt:api-ms-win-crt-heap-l1-1-0.dll
 0002:0000493c       __IMPORT_DESCRIPTOR_api-ms-win-crt-runtime-l1-1-0 1000c93c     ucrt:api-ms-win-crt-runtime-l1-1-0.dll
 0002:00004950       __NULL_IMPORT_DESCRIPTOR   1000c950     kernel32:KERNEL32.dll
 0003:00000000       ___security_cookie_complement 1000d000     MSVCRT:gs_cookie.obj
 0003:00000004       ___security_cookie         1000d004     MSVCRT:gs_cookie.obj
 0003:00000010       ___scrt_native_dllmain_reason 1000d010     MSVCRT:utility.obj
 0003:00000020       ___isa_enabled             1000d020     MSVCRT:cpu_disp.obj
 0003:00000024       ___scrt_ucrt_dll_is_in_use 1000d024     MSVCRT:ucrt_stubs.obj
 0003:00000028       ??_R0?AVbad_alloc@std@@@8  1000d028     AccessBridgeMessageQueue.obj
 0003:00000044       ??_R0?AVexception@std@@@8  1000d044     AccessBridgeMessageQueue.obj
 0003:00000060       ??_R0?AVbad_array_new_length@std@@@8 1000d060     MSVCRT:throw_bad_alloc.obj
 0003:00000088       ??_R0?AVtype_info@@@8      1000d088     MSVCRT:std_type_info_static.obj
 0003:000000a0       ?_OptionsStorage@?1??__local_stdio_printf_options@@9@4_KA 1000d0a0     AccessBridgeDebug.obj
 0003:000000ac       ?theFromJavaHelloMsgID@@3IA 1000d0ac     AccessBridgeMessages.obj
 0003:000000b0       ?theFromWindowsHelloMsgID@@3IA 1000d0b0     AccessBridgeMessages.obj
 0003:000000b4       ?sendMemoryIPCLock@@3U_RTL_CRITICAL_SECTION@@A 1000d0b4     WinAccessBridge.obj
 0003:000000cc       ?newJVMs@@3PAPADA          1000d0cc     WinAccessBridge.obj
 0003:000000d0       ?theWindowsAccessBridge@@3PAVWinAccessBridge@@A 1000d0d0     WinAccessBridge.obj
 0003:000000d4       ?theDialogWindow@@3PAUHWND__@@A 1000d0d4     WinAccessBridge.obj
 0003:000000d8       ?isVMInstanceChainInUse@@3_NA 1000d0d8     WinAccessBridge.obj
 0003:00000400       ?__type_info_root_node@@3U__type_info_node@@A 1000d400     MSVCRT:tncleanup.obj
 0003:00000408       ?_OptionsStorage@?1??__local_stdio_scanf_options@@9@4_KA 1000d408     MSVCRT:default_local_stdio_options.obj
 0003:00000410       ___scrt_current_native_startup_state 1000d410     MSVCRT:utility.obj
 0003:00000414       ___scrt_native_startup_lock 1000d414     MSVCRT:utility.obj
 0003:00000434       ___scrt_debugger_hook_flag 1000d434     MSVCRT:utility_desktop.obj
 0003:00000438       ___isa_available           1000d438     MSVCRT:cpu_disp.obj
 0003:0000043c       ___favor                   1000d43c     MSVCRT:cpu_disp.obj
 0003:00000440       ___dyn_tls_init_callback   1000d440     <common>

 entry point at        0001:00005bdb

 Static symbols

 0000:ffff0000       .debug$S                   10000000     windowsaccessbridge.exp
 0000:ffff0000       .debug$S                   10000000     vcruntime:VCRUNTIME140.dll
 0000:ffff0000       .debug$S                   10000000     vcruntime:VCRUNTIME140.dll
 0000:ffff0000       .debug$S                   10000000     vcruntime:VCRUNTIME140.dll
 0000:ffff0000       .debug$S                   10000000     vcruntime:VCRUNTIME140.dll
 0000:ffff0000       .debug$S                   10000000     vcruntime:VCRUNTIME140.dll
 0000:ffff0000       .debug$S                   10000000     vcruntime:VCRUNTIME140.dll
 0000:ffff0000       .debug$S                   10000000     vcruntime:VCRUNTIME140.dll
 0000:ffff0000       .debug$S                   10000000     vcruntime:VCRUNTIME140.dll
 0000:ffff0000       .debug$S                   10000000     vcruntime:VCRUNTIME140.dll
 0000:ffff0000       .debug$S                   10000000     ucrt:api-ms-win-crt-environment-l1-1-0.dll
 0000:ffff0000       .debug$S                   10000000     ucrt:api-ms-win-crt-heap-l1-1-0.dll
 0000:ffff0000       .debug$S                   10000000     ucrt:api-ms-win-crt-heap-l1-1-0.dll
 0000:ffff0000       .debug$S                   10000000     ucrt:api-ms-win-crt-heap-l1-1-0.dll
 0000:ffff0000       .debug$S                   10000000     ucrt:api-ms-win-crt-runtime-l1-1-0.dll
 0000:ffff0000       .debug$S                   10000000     ucrt:api-ms-win-crt-runtime-l1-1-0.dll
 0000:ffff0000       .debug$S                   10000000     ucrt:api-ms-win-crt-runtime-l1-1-0.dll
 0000:ffff0000       .debug$S                   10000000     ucrt:api-ms-win-crt-runtime-l1-1-0.dll
 0000:ffff0000       .debug$S                   10000000     ucrt:api-ms-win-crt-runtime-l1-1-0.dll
 0000:ffff0000       .debug$S                   10000000     ucrt:api-ms-win-crt-runtime-l1-1-0.dll
 0000:ffff0000       .debug$S                   10000000     ucrt:api-ms-win-crt-runtime-l1-1-0.dll
 0000:ffff0000       .debug$S                   10000000     ucrt:api-ms-win-crt-runtime-l1-1-0.dll
 0000:ffff0000       .debug$S                   10000000     ucrt:api-ms-win-crt-runtime-l1-1-0.dll
 0000:ffff0000       .debug$S                   10000000     ucrt:api-ms-win-crt-runtime-l1-1-0.dll
 0000:ffff0000       .debug$S                   10000000     ucrt:api-ms-win-crt-runtime-l1-1-0.dll
 0000:ffff0000       .debug$S                   10000000     ucrt:api-ms-win-crt-runtime-l1-1-0.dll
 0000:ffff0000       .debug$S                   10000000     ucrt:api-ms-win-crt-stdio-l1-1-0.dll
 0000:ffff0000       .debug$S                   10000000     ucrt:api-ms-win-crt-stdio-l1-1-0.dll
 0000:ffff0000       .debug$S                   10000000     ucrt:api-ms-win-crt-stdio-l1-1-0.dll
 0000:ffff0000       .debug$S                   10000000     ucrt:api-ms-win-crt-stdio-l1-1-0.dll
 0000:ffff0000       .debug$S                   10000000     ucrt:api-ms-win-crt-stdio-l1-1-0.dll
 0000:ffff0000       .debug$S                   10000000     ucrt:api-ms-win-crt-stdio-l1-1-0.dll
 0000:ffff0000       .debug$S                   10000000     ucrt:api-ms-win-crt-string-l1-1-0.dll
 0000:ffff0000       .debug$S                   10000000     ucrt:api-ms-win-crt-string-l1-1-0.dll
 0000:ffff0000       .debug$S                   10000000     ucrt:api-ms-win-crt-string-l1-1-0.dll
 0000:ffff0000       .debug$S                   10000000     ucrt:api-ms-win-crt-string-l1-1-0.dll
 0000:ffff0000       .debug$S                   10000000     ucrt:api-ms-win-crt-string-l1-1-0.dll
 0000:ffff0000       .debug$S                   10000000     ucrt:api-ms-win-crt-string-l1-1-0.dll
 0000:ffff0000       .debug$S                   10000000     kernel32:KERNEL32.dll
 0000:ffff0000       .debug$S                   10000000     kernel32:KERNEL32.dll
 0000:ffff0000       .debug$S                   10000000     kernel32:KERNEL32.dll
 0000:ffff0000       .debug$S                   10000000     kernel32:KERNEL32.dll
 0000:ffff0000       .debug$S                   10000000     kernel32:KERNEL32.dll
 0000:ffff0000       .debug$S                   10000000     kernel32:KERNEL32.dll
 0000:ffff0000       .debug$S                   10000000     kernel32:KERNEL32.dll
 0000:ffff0000       .debug$S                   10000000     kernel32:KERNEL32.dll
 0000:ffff0000       .debug$S                   10000000     kernel32:KERNEL32.dll
 0000:ffff0000       .debug$S                   10000000     kernel32:KERNEL32.dll
 0000:ffff0000       .debug$S                   10000000     kernel32:KERNEL32.dll
 0000:ffff0000       .debug$S                   10000000     kernel32:KERNEL32.dll
 0000:ffff0000       .debug$S                   10000000     kernel32:KERNEL32.dll
 0000:ffff0000       .debug$S                   10000000     kernel32:KERNEL32.dll
 0000:ffff0000       .debug$S                   10000000     kernel32:KERNEL32.dll
 0000:ffff0000       .debug$S                   10000000     kernel32:KERNEL32.dll
 0000:ffff0000       .debug$S                   10000000     kernel32:KERNEL32.dll
 0000:ffff0000       .debug$S                   10000000     kernel32:KERNEL32.dll
 0000:ffff0000       .debug$S                   10000000     kernel32:KERNEL32.dll
 0000:ffff0000       .debug$S                   10000000     kernel32:KERNEL32.dll
 0000:ffff0000       .debug$S                   10000000     kernel32:KERNEL32.dll
 0000:ffff0000       .debug$S                   10000000     kernel32:KERNEL32.dll
 0000:ffff0000       .debug$S                   10000000     kernel32:KERNEL32.dll
 0000:ffff0000       .debug$S                   10000000     kernel32:KERNEL32.dll
 0000:ffff0000       .debug$S                   10000000     user32:USER32.dll
 0000:ffff0000       .debug$S                   10000000     user32:USER32.dll
 0000:ffff0000       .debug$S                   10000000     user32:USER32.dll
 0000:ffff0000       .debug$S                   10000000     user32:USER32.dll
 0000:ffff0000       .debug$S                   10000000     user32:USER32.dll
 0000:ffff0000       .debug$S                   10000000     user32:USER32.dll
 0000:ffff0000       .debug$S                   10000000     user32:USER32.dll
 0000:ffff0000       .debug$S                   10000000     user32:USER32.dll
 0000:ffff0000       .debug$S                   10000000     user32:USER32.dll
 0000:ffff0000       .debug$S                   10000000     user32:USER32.dll
 0000:ffff0000       .debug$S                   10000000     user32:USER32.dll
 0000:ffff0000       .debug$S                   10000000     user32:USER32.dll
 0000:ffff0000       .debug$S                   10000000     user32:USER32.dll
 0001:00005790       $$000000                   10006790     MSVCRT:ulldiv.obj
 0001:000057b2       L1                         100067b2     MSVCRT:ulldiv.obj
 0001:000057c0       L3                         100067c0     MSVCRT:ulldiv.obj
 0001:000057ee       L4                         100067ee     MSVCRT:ulldiv.obj
 0001:000057ef       L5                         100067ef     MSVCRT:ulldiv.obj
 0001:000057f3       L2                         100067f3     MSVCRT:ulldiv.obj
 0001:00005870       $$000000                   10006870     MSVCRT:chkstk.obj
 0001:00005884       cs10                       10006884     MSVCRT:chkstk.obj
 0001:00005892       cs20                       10006892     MSVCRT:chkstk.obj
 0001:0000589b       ?dllmain_crt_dispatch@@YGHQAUHINSTANCE__@@KQAX@Z 1000689b f   MSVCRT:dll_dllmain.obj
 0001:000058ee       ?dllmain_crt_process_attach@@YAHQAUHINSTANCE__@@QAX@Z 100068ee f   MSVCRT:dll_dllmain.obj
 0001:000059f5       ?dllmain_crt_process_detach@@YAH_N@Z 100069f5 f   MSVCRT:dll_dllmain.obj
 0001:00005aa5       ?dllmain_dispatch@@YAHQAUHINSTANCE__@@KQAX@Z 10006aa5 f   MSVCRT:dll_dllmain.obj
 0001:00005bb0       ?dllmain_raw@@YGHQAUHINSTANCE__@@KQAX@Z 10006bb0 f   MSVCRT:dll_dllmain.obj
 0001:00005dbf       ___get_entropy             10006dbf f   MSVCRT:gs_support.obj
 0001:00005e92       ?find_pe_section@@YAPAU_IMAGE_SECTION_HEADER@@QAEI@Z 10006e92 f   MSVCRT:utility.obj
 0001:000062f0       $$000000                   100072f0     MSVCRT:sehprolg4.obj
 0002:00003340       _GS_ExceptionPointers      1000b340     MSVCRT:gs_report.obj
 0002:000039a8       __sehtable$?dllmain_crt_process_attach@@YAHQAUHINSTANCE__@@QAX@Z 1000b9a8     MSVCRT:dll_dllmain.obj
 0002:000039c8       __sehtable$?dllmain_crt_process_detach@@YAH_N@Z 1000b9c8     MSVCRT:dll_dllmain.obj
 0002:000039f0       __sehtable$?dllmain_dispatch@@YAHQAUHINSTANCE__@@KQAX@Z 1000b9f0     MSVCRT:dll_dllmain.obj
 0002:00003a48       __sehtable$___scrt_is_nonwritable_in_current_image 1000ba48     MSVCRT:utility.obj
 0002:00003a70       .edata                     1000ba70     windowsaccessbridge.exp
 0002:00003a98       rgpv                       1000ba98     windowsaccessbridge.exp
 0002:00003c2c       rgszName                   1000bc2c     windowsaccessbridge.exp
 0002:00003dc0       rgwOrd                     1000bdc0     windowsaccessbridge.exp
 0002:00003e8a       szName                     1000be8a     windowsaccessbridge.exp
 0002:00003ea2       $N00001                    1000bea2     windowsaccessbridge.exp
 0002:00003ec4       $N00002                    1000bec4     windowsaccessbridge.exp
 0002:00003edd       $N00003                    1000bedd     windowsaccessbridge.exp
 0002:00003f02       $N00004                    1000bf02     windowsaccessbridge.exp
 0002:00003f1e       $N00005                    1000bf1e     windowsaccessbridge.exp
 0002:00003f2a       $N00006                    1000bf2a     windowsaccessbridge.exp
 0002:00003f46       $N00007                    1000bf46     windowsaccessbridge.exp
 0002:00003f68       $N00008                    1000bf68     windowsaccessbridge.exp
 0002:00003f8c       $N00009                    1000bf8c     windowsaccessbridge.exp
 0002:00003fa0       $N00010                    1000bfa0     windowsaccessbridge.exp
 0002:00003fb5       $N00011                    1000bfb5     windowsaccessbridge.exp
 0002:00003fd3       $N00012                    1000bfd3     windowsaccessbridge.exp
 0002:00003fea       $N00013                    1000bfea     windowsaccessbridge.exp
 0002:00004007       $N00014                    1000c007     windowsaccessbridge.exp
 0002:00004020       $N00015                    1000c020     windowsaccessbridge.exp
 0002:0000403e       $N00016                    1000c03e     windowsaccessbridge.exp
 0002:00004055       $N00017                    1000c055     windowsaccessbridge.exp
 0002:00004071       $N00018                    1000c071     windowsaccessbridge.exp
 0002:00004088       $N00019                    1000c088     windowsaccessbridge.exp
 0002:000040a2       $N00020                    1000c0a2     windowsaccessbridge.exp
 0002:000040c2       $N00021                    1000c0c2     windowsaccessbridge.exp
 0002:000040d5       $N00022                    1000c0d5     windowsaccessbridge.exp
 0002:000040ee       $N00023                    1000c0ee     windowsaccessbridge.exp
 0002:0000410d       $N00024                    1000c10d     windowsaccessbridge.exp
 0002:00004126       $N00025                    1000c126     windowsaccessbridge.exp
 0002:0000414d       $N00026                    1000c14d     windowsaccessbridge.exp
 0002:0000416f       $N00027                    1000c16f     windowsaccessbridge.exp
 0002:0000418a       $N00028                    1000c18a     windowsaccessbridge.exp
 0002:000041a3       $N00029                    1000c1a3     windowsaccessbridge.exp
 0002:000041c7       $N00030                    1000c1c7     windowsaccessbridge.exp
 0002:000041e6       $N00031                    1000c1e6     windowsaccessbridge.exp
 0002:0000420d       $N00032                    1000c20d     windowsaccessbridge.exp
 0002:00004230       $N00033                    1000c230     windowsaccessbridge.exp
 0002:00004248       $N00034                    1000c248     windowsaccessbridge.exp
 0002:0000425f       $N00035                    1000c25f     windowsaccessbridge.exp
 0002:00004275       $N00036                    1000c275     windowsaccessbridge.exp
 0002:00004296       $N00037                    1000c296     windowsaccessbridge.exp
 0002:000042b2       $N00038                    1000c2b2     windowsaccessbridge.exp
 0002:000042d6       $N00039                    1000c2d6     windowsaccessbridge.exp
 0002:000042f6       $N00040                    1000c2f6     windowsaccessbridge.exp
 0002:00004312       $N00041                    1000c312     windowsaccessbridge.exp
 0002:00004328       $N00042                    1000c328     windowsaccessbridge.exp
 0002:0000433f       $N00043                    1000c33f     windowsaccessbridge.exp
 0002:0000435b       $N00044                    1000c35b     windowsaccessbridge.exp
 0002:00004372       $N00045                    1000c372     windowsaccessbridge.exp
 0002:00004388       $N00046                    1000c388     windowsaccessbridge.exp
 0002:000043a7       $N00047                    1000c3a7     windowsaccessbridge.exp
 0002:000043bb       $N00048                    1000c3bb     windowsaccessbridge.exp
 0002:000043cc       $N00049                    1000c3cc     windowsaccessbridge.exp
 0002:000043f1       $N00050                    1000c3f1     windowsaccessbridge.exp
 0002:00004402       $N00051                    1000c402     windowsaccessbridge.exp
 0002:0000441f       $N00052                    1000c41f     windowsaccessbridge.exp
 0002:00004444       $N00053                    1000c444     windowsaccessbridge.exp
 0002:00004469       $N00054                    1000c469     windowsaccessbridge.exp
 0002:00004478       $N00055                    1000c478     windowsaccessbridge.exp
 0002:0000448a       $N00056                    1000c48a     windowsaccessbridge.exp
 0002:000044a4       $N00057                    1000c4a4     windowsaccessbridge.exp
 0002:000044bd       $N00058                    1000c4bd     windowsaccessbridge.exp
 0002:000044cf       $N00059                    1000c4cf     windowsaccessbridge.exp
 0002:000044de       $N00060                    1000c4de     windowsaccessbridge.exp
 0002:000044f7       $N00061                    1000c4f7     windowsaccessbridge.exp
 0002:0000450a       $N00062                    1000c50a     windowsaccessbridge.exp
 0002:00004522       $N00063                    1000c522     windowsaccessbridge.exp
 0002:00004547       $N00064                    1000c547     windowsaccessbridge.exp
 0002:00004567       $N00065                    1000c567     windowsaccessbridge.exp
 0002:00004584       $N00066                    1000c584     windowsaccessbridge.exp
 0002:00004591       $N00067                    1000c591     windowsaccessbridge.exp
 0002:0000459e       $N00068                    1000c59e     windowsaccessbridge.exp
 0002:000045b0       $N00069                    1000c5b0     windowsaccessbridge.exp
 0002:000045d5       $N00070                    1000c5d5     windowsaccessbridge.exp
 0002:000045e2       $N00071                    1000c5e2     windowsaccessbridge.exp
 0002:0000460a       $N00072                    1000c60a     windowsaccessbridge.exp
 0002:0000461a       $N00073                    1000c61a     windowsaccessbridge.exp
 0002:0000462b       $N00074                    1000c62b     windowsaccessbridge.exp
 0002:0000463c       $N00075                    1000c63c     windowsaccessbridge.exp
 0002:0000464d       $N00076                    1000c64d     windowsaccessbridge.exp
 0002:0000465c       $N00077                    1000c65c     windowsaccessbridge.exp
 0002:0000466e       $N00078                    1000c66e     windowsaccessbridge.exp
 0002:00004680       $N00079                    1000c680     windowsaccessbridge.exp
 0002:00004694       $N00080                    1000c694     windowsaccessbridge.exp
 0002:000046a6       $N00081                    1000c6a6     windowsaccessbridge.exp
 0002:000046b8       $N00082                    1000c6b8     windowsaccessbridge.exp
 0002:000046ca       $N00083                    1000c6ca     windowsaccessbridge.exp
 0002:000046db       $N00084                    1000c6db     windowsaccessbridge.exp
 0002:000046ed       $N00085                    1000c6ed     windowsaccessbridge.exp
 0002:00004700       $N00086                    1000c700     windowsaccessbridge.exp
 0002:00004717       $N00087                    1000c717     windowsaccessbridge.exp
 0002:00004739       $N00088                    1000c739     windowsaccessbridge.exp
 0002:00004759       $N00089                    1000c759     windowsaccessbridge.exp
 0002:0000477d       $N00090                    1000c77d     windowsaccessbridge.exp
 0002:00004796       $N00091                    1000c796     windowsaccessbridge.exp
 0002:000047aa       $N00092                    1000c7aa     windowsaccessbridge.exp
 0002:000047c3       $N00093                    1000c7c3     windowsaccessbridge.exp
 0002:000047e2       $N00094                    1000c7e2     windowsaccessbridge.exp
 0002:000047fa       $N00095                    1000c7fa     windowsaccessbridge.exp
 0002:00004817       $N00096                    1000c817     windowsaccessbridge.exp
 0002:00004830       $N00097                    1000c830     windowsaccessbridge.exp
 0002:0000484e       $N00098                    1000c84e     windowsaccessbridge.exp
 0002:00004866       $N00099                    1000c866     windowsaccessbridge.exp
 0002:0000487f       $N00100                    1000c87f     windowsaccessbridge.exp
 0002:0000489e       $N00101                    1000c89e     windowsaccessbridge.exp
 0002:00004b28       .idata$6                   1000cb28     kernel32:KERNEL32.dll
 0002:00004be4       .idata$6                   1000cbe4     user32:USER32.dll
 0002:00004c86       .idata$6                   1000cc86     vcruntime:VCRUNTIME140.dll
 0002:00004df0       .idata$6                   1000cdf0     ucrt:api-ms-win-crt-string-l1-1-0.dll
 0002:00004e12       .idata$6                   1000ce12     ucrt:api-ms-win-crt-stdio-l1-1-0.dll
 0002:00004e32       .idata$6                   1000ce32     ucrt:api-ms-win-crt-environment-l1-1-0.dll
 0002:00004e58       .idata$6                   1000ce58     ucrt:api-ms-win-crt-heap-l1-1-0.dll
 0002:00004e78       .idata$6                   1000ce78     ucrt:api-ms-win-crt-runtime-l1-1-0.dll
 0003:000000a8       _logFP                     1000d0a8     AccessBridgeDebug.obj
 0003:000000dc       ?__proc_attached@@3HA      1000d0dc     MSVCRT:dll_dllmain.obj
 0003:000000e0       _GS_ExceptionRecord        1000d0e0     MSVCRT:gs_report.obj
 0003:00000130       _GS_ContextRecord          1000d130     MSVCRT:gs_report.obj
 0003:00000418       ?is_initialized_as_dll@@3_NA 1000d418     MSVCRT:utility.obj
 0003:00000419       ?module_local_atexit_table_initialized@@3_NA 1000d419     MSVCRT:utility.obj
 0003:0000041c       ?module_local_atexit_table@@3U_onexit_table_t@@A 1000d41c     MSVCRT:utility.obj
 0003:00000428       ?module_local_at_quick_exit_table@@3U_onexit_table_t@@A 1000d428     MSVCRT:utility.obj
 0004:00000120       $R000000                   1000e120     windowsaccessbridge.dll.res
 0004:000004b8       $R000398                   1000e4b8     windowsaccessbridge.dll.res
 0004:000006d0       $R0005B0                   1000e6d0     windowsaccessbridge.dll.res
